:020000040000FA
:0408000098EF0BF072
:1008100003B275EF05F0F2B493EF05F09EB09BEFD5
:1008200005F09EB2A3EF05F0F2A81AEF04F0F2B2C1
:1008300023EF04F0F2B01FEF04F047EF0BF0F29655
:10084000F29047EF0BF0CD90F2929EA02DEF04F0C6
:100850000101533F2DEF04F0542BB2C1B6F1B3C1E7
:10086000B7F1B4C1B8F1B5C1B9F1AEC1B2F1AFC120
:10087000B3F1B0C1B4F1B1C1B5F1AAC1AEF1ABC130
:10088000AFF1ACC1B0F1ADC1B1F1A6C1AAF1A7C140
:10089000ABF1A8C1ACF1A9C1ADF1A2C1A6F1A3C150
:1008A000A7F1A4C1A8F1A5C1A9F19EC1A2F19FC160
:1008B000A3F1A0C1A4F1A1C1A5F19AC19EF19BC170
:1008C0009FF19CC1A0F19DC1A1F1CECF9AF1CFCFF4
:1008D0009BF153C19CF154C19DF1CF6ACE6A0101D5
:1008E000536B546B9E90CD800FBC0F8E0FBA7CEF74
:1008F00004F00F8A47EF0BF013880F8C0FBEB9EF8F
:1009000004F09AC19EF19BC19FF19CC1A0F19DC1D1
:10091000A1F19EC1A2F19FC1A3F1A0C1A4F1A1C107
:10092000A5F1A2C1A6F1A3C1A7F1A4C1A8F1A5C1D7
:10093000A9F1A6C1AAF1A7C1ABF1A8C1ACF1A9C1A7
:10094000ADF1AAC1AEF1ABC1AFF1ACC1B0F1ADC177
:10095000B1F1AEC1B2F1AFC1B3F1B0C1B4F1B1C147
:10096000B5F1B2C1B6F1B3C1B7F1B4C1B8F1B5C117
:10097000B9F101015E6B5F6B606B616B9A515E2731
:100980009B515F239C5160239D5161239E515E27A3
:100990009F515F23A0516023A1516123A2515E2783
:1009A000A3515F23A4516023A5516123A6515E2763
:1009B000A7515F23A8516023A9516123AA515E2743
:1009C000AB515F23AC516023AD516123AE515E2723
:1009D000AF515F23B0516023B1516123B2515E2703
:1009E000B3515F23B4516023B5516123B6515E27E3
:1009F000B7515F23B8516023B9516123D8900101E9
:100A0000613360335F335E33D8900101613360330B
:100A10005F335E33D8900101613360335F335E33FF
:100A200000C10CF101C10DF102C10EF103C10FF1C2
:100A300004C110F105C111F106C112F107C113F192
:100A400008C114F109C115F10AC116F10BC117F162
:100A500034C135F111B838EF05F00101620E046FB1
:100A6000010E056F000E066F000E076F41EF05F0D7
:100A70000101A70E046F020E056F000E066F000E37
:100A8000076F5EC100F15FC101F160C102F161C198
:100A900003F185EC2FF003BF04D01CBE02D01CA0D4
:100AA000108C11A059EF05F010BA59EF05F00F8026
:100AB000108A0CC100F10DC101F10EC102F10FC18C
:100AC00003F110C104F111C105F112C106F113C106
:100AD00007F114C108F115C109F116C10AF117C1D6
:100AE0000BF135C134F147EF0BF00392ABB2AB9889
:100AF000AB88030103EE00F080517F0BE92604C0B0
:100B0000EFFF802B8151805D700BD8A48B82000099
:100B10008051815D700BD8A48B9281518019D8B41B
:100B2000079047EF0BF0F2940101453F47EF0BF0C0
:100B3000462B47EF0BF09E900101533F47EF0BF020
:100B4000542B47EF0BF09E9211B843EF08F00400CE
:100B500066A1ABEF05F08BB4B5EF05F010ACB5EFC7
:100B600005F08B84109CB6EF05F08B94077C07ACE6
:100B7000D1EF05F0C274C2B4CBEF05F0C3CFB7F527
:100B8000C4CFB8F50501D890B833B733D890B8338F
:100B9000B733D2EF05F0C3CF55F1C4CF56F1D2EF42
:100BA00005F0C28207B444EF06F047C14BF148C1DB
:100BB0004CF149C14DF14AC14EF15EC162F15FC1D4
:100BC00063F160C164F161C165F113A8EAEF05F05A
:100BD000138C13989AC1BAF19BC1BBF19CC1BCF1B3
:100BE0009DC1BDF19EC1BEF19FC1BFF1A0C1C0F1C9
:100BF000A1C1C1F1A2C1C2F1A3C1C3F1A4C1C4F199
:100C0000A5C1C5F1A6C1C6F1A7C1C7F1A8C1C8F168
:100C1000A9C1C9F1AAC1CAF1ABC1CBF1ACC1CCF138
:100C2000ADC1CDF1AEC1CEF1AFC1CFF1B0C1D0F108
:100C3000B1C1D1F1B2C1D2F1B3C1D3F1B4C1D4F1D8
:100C4000B5C1D5F1B6C1D6F1B7C1D7F1B8C1D8F1A8
:100C5000B9C1D9F1B7C5B9F5B8C5BAF5B9C5BBF5CC
:100C6000BAC5BCF5010155515B2756515C23E86AB2
:100C70005D230E2E44EF06F05CC157F15DC158F1C3
:100C80005B6B5C6B5D6B078E0201002F47EF0BF017
:100C90003C0E006F1D50E00BE00AE86612881BBE98
:100CA00002D01BB4108E00C10CF101C10DF102C1C4
:100CB0000EF103C10FF104C110F105C111F106C11C
:100CC00012F107C113F108C114F109C115F10AC1EC
:100CD00016F10BC117F134C135F181AAACEF06F062
:100CE00015A4F7EF06F005012F51000AD8B43AEF2A
:100CF00007F005012F51010AD8B4B6EF06F005013F
:100D00002F51020AD8B4F7EF06F005012F51030A5C
:100D1000D8B4F7EF06F005012F51040AD8B4F7EF65
:100D200006F005012F51050AD8B4F7EF06F00501CA
:100D30002F51060AD8B4F7EF06F005012F51070A24
:100D4000D8B4F7EF06F005012F51320AD8B4B4EF4A
:100D500006F02F6B3AEF07F000011650030AD8B4E3
:100D6000F7EF06F03AEF07F03AEF07F005015767A3
:100D7000C1EF06F05867C1EF06F05967C1EF06F002
:100D80005A67C5EF06F03AEF07F05BC500F15CC5A6
:100D900001F15DC502F15EC503F10101010E046FB1
:100DA000000E056F000E066F000E076F85EC2FF02A
:100DB00000C15BF501C15CF502C15DF503C15EF5E3
:100DC00001010067EBEF06F00167EBEF06F0026749
:100DD000EBEF06F003673AEF07F057C55BF558C530
:100DE0005CF559C55DF55AC55EF524EF07F00FBEF9
:100DF0000CEF07F010A011EF07F00101476708EFB3
:100E000007F0486708EF07F0496708EF07F04A67FF
:100E10000CEF07F011EF07F007AE11EF07F024EF2A
:100E200007F00501312F3AEF07F03C0E316F302FFC
:100E30003AEF07F00101000E626FE00E636FA50E3E
:100E4000646F010E656F138800011650000AD8B454
:100E500032EF07F000011650030AD8B437EF07F05D
:100E60003AEF07F00001010E166E3AEF07F00001AD
:100E7000040E166E0501666B37B740EF07F066810A
:100E80000CC100F10DC101F10EC102F10FC103F15E
:100E900010C104F111C105F112C106F113C107F12E
:100EA00014C108F115C109F116C10AF117C10BF1FE
:100EB00035C134F100C10CF101C10DF102C10EF1D7
:100EC00003C10FF104C110F105C111F106C112F106
:100ED00007C113F108C114F109C115F10AC116F1D6
:100EE0000BC117F134C135F101018E677FEF07F0B7
:100EF0008F677FEF07F090677FEF07F0916783EFD1
:100F000007F0B4EF07F092C100F193C101F194C171
:100F100002F195C103F10101010E046F000E056F8E
:100F2000000E066F000E076F85EC2FF000C192F1E6
:100F300001C193F102C194F103C195F10101006770
:100F4000A9EF07F00167A9EF07F00267A9EF07F023
:100F50000367B4EF07F08EC192F18FC193F190C196
:100F600094F191C195F10F80D57ED5BE6ED0D6CFCC
:100F700047F1D7CF48F145C149F1E86AE8CF4AF1D6
:100F8000138A1CBE02D01CA0108C109047C100F127
:100F900048C101F149C102F14AC103F101010A0E40
:100FA000046F000E056F000E066F000E076F85ECD4
:100FB0002FF003AF1080010154A7EBEF07F00F9A59
:100FC0000F9C0F9E0101000E5E6F600E5F6F3D0E65
:100FD000606F080E616F010147BFFBEF07F04867C4
:100FE000FBEF07F04967FBEF07F04A67FBEF07F0FD
:100FF000F28820EF08F0F2985E6B5F6B606B616BBC
:101000009A6B9B6B9C6B9D6B9E6B9F6BA06BA16B9C
:10101000A26BA36BA46BA56BA66BA76BA86BA96B4C
:10102000AA6BAB6BAC6BAD6BAE6BAF6BB06BB16BFC
:10103000B26BB36BB46BB56BB66BB76BB86BB96BAC
:10104000D76AD66A0101456B466B0CC100F10DC130
:1010500001F10EC102F10FC103F110C104F111C180
:1010600005F112C106F113C107F114C108F115C150
:1010700009F116C10AF117C10BF135C134F147EF7F
:101080000BF047EF0BF00201002FABEF0AF0D59EFB
:10109000D6CF47F1D7CF48F145C149F1E86AE8CF4B
:1010A0004AF1138AD76AD66A0101456B466BD58E21
:1010B0001D50E00BE00AE86612881BBE02D01BB48C
:1010C000108E1AAE1F8C00C10CF101C10DF102C1CE
:1010D0000EF103C10FF104C110F105C111F106C1F8
:1010E00012F107C113F108C114F109C115F10AC1C8
:1010F00016F10BC117F134C135F10FA0109A11B8D8
:101100008DEF08F00101620E046F010E056F000EF5
:10111000066F000E076F96EF08F00101A70E046F2F
:10112000020E056F000E066F000E076F47C100F13B
:1011300048C101F149C102F14AC103F185EC2FF028
:1011400003BFA9EF08F01CBE02D01CA0108C11B088
:101150000F800CC100F10DC101F10EC102F10FC1F0
:1011600003F110C104F111C105F112C106F113C15F
:1011700007F114C108F115C109F116C10AF117C12F
:101180000BF135C134F102013C0E006F00C10CF1CE
:1011900001C10DF102C10EF103C10FF104C110F143
:1011A00005C111F106C112F107C113F108C114F113
:1011B00009C115F10AC116F10BC117F134C135F19E
:1011C00081BAE6EF08F015B225EF09F015A025EF7A
:1011D00009F015A470EF09F005012F51000AD8B4E9
:1011E000B3EF09F005012F51010AD8B42FEF09F030
:1011F00005012F51020AD8B470EF09F005012F51F3
:10120000030AD8B470EF09F005012F51040AD8B4CD
:1012100070EF09F005012F51050AD8B470EF09F0FD
:1012200005012F51060AD8B470EF09F005012F51BE
:10123000070AD8B470EF09F005012F51320AD8B46B
:101240002DEF09F02F6BB3EF09F000011650030AE0
:10125000D8B470EF09F0B3EF09F0B3EF09F005016E
:1012600057673AEF09F058673AEF09F059673AEFD4
:1012700009F05A673EEF09F0B3EF09F05BC500F1E2
:101280005CC501F15DC502F15EC503F10101010E0E
:10129000046F000E056F000E066F000E076F85ECE1
:1012A0002FF000C15BF501C15CF502C15DF503C122
:1012B0005EF50101006764EF09F0016764EF09F072
:1012C000026764EF09F00367B3EF09F057C55BF5F8
:1012D00058C55CF559C55DF55AC55EF59DEF09F039
:1012E0000FBE85EF09F010A08AEF09F001014767F2
:1012F00081EF09F0486781EF09F0496781EF09F054
:101300004A6785EF09F08AEF09F007AE8AEF09F026
:101310009DEF09F00501312FB3EF09F03C0E316F5D
:10132000302FB3EF09F00101000E626FE00E636F22
:10133000A50E646F010E656F138800011650000A38
:10134000D8B4ABEF09F000011650030AD8B4B0EFDF
:1013500009F0B3EF09F00001010E166EB3EF09F0CA
:101360000001040E166E0501666B37B7B9EF09F080
:1013700066810CC100F10DC101F10EC102F10FC176
:1013800003F110C104F111C105F112C106F113C13D
:1013900007F114C108F115C109F116C10AF117C10D
:1013A0000BF135C134F100C10CF101C10DF102C1E5
:1013B0000EF103C10FF104C110F105C111F106C115
:1013C00012F107C113F108C114F109C115F10AC1E5
:1013D00016F10BC117F134C135F101018E67F8EF39
:1013E00009F08F67F8EF09F09067F8EF09F091675F
:1013F000FCEF09F02DEF0AF092C100F193C101F169
:1014000094C102F195C103F10101010E046F000EB8
:10141000056F000E066F000E076F85EC2FF000C100
:1014200092F101C193F102C194F103C195F101015F
:10143000006722EF0AF0016722EF0AF0026722EF4D
:101440000AF003672DEF0AF08EC192F18FC193F17C
:1014500090C194F191C195F10F80109047C100F1B6
:1014600048C101F149C102F14AC103F101010A0E6B
:10147000046F000E056F000E066F000E076F85ECFF
:101480002FF003AF1080010154A753EF0AF00F9A19
:101490000F9C0F9E0101000E5E6F600E5F6F3D0E90
:1014A000606F080E616F47C100F148C101F149C189
:1014B00002F14AC103F10101140E046F050E056F1C
:1014C000000E066F000E076F85EC2FF003AF6CEF78
:1014D0000AF0F28891EF0AF0F2985E6B5F6B606B36
:1014E000616B9A6B9B6B9C6B9D6B9E6B9F6BA06BF8
:1014F000A16BA26BA36BA46BA56BA66BA76BA86B70
:10150000A96BAA6BAB6BAC6BAD6BAE6BAF6BB06B1F
:10151000B16BB26BB36BB46BB56BB66BB76BB86BCF
:10152000B96B0CC100F10DC101F10EC102F10FC187
:1015300003F110C104F111C105F112C106F113C18B
:1015400007F114C108F115C109F116C10AF117C15B
:101550000BF135C134F104008BB4B6EF0AF010ACD6
:10156000B6EF0AF08B84109CB7EF0AF08B94077CDF
:1015700007ACD2EF0AF0C274C2B4CCEF0AF0C3CF0A
:10158000B7F5C4CFB8F50501D890B833B733D890C4
:10159000B833B733D3EF0AF0C3CF55F1C4CF56F108
:1015A000D3EF0AF0C28207B445EF0BF047C14BF10D
:1015B00048C14CF149C14DF14AC14EF15EC162F1E1
:1015C0005FC163F160C164F161C165F113A8EBEF24
:1015D0000AF0138C13989AC1BAF19BC1BBF19CC15C
:1015E000BCF19DC1BDF19EC1BEF19FC1BFF1A0C1C3
:1015F000C0F1A1C1C1F1A2C1C2F1A3C1C3F1A4C193
:10160000C4F1A5C1C5F1A6C1C6F1A7C1C7F1A8C162
:10161000C8F1A9C1C9F1AAC1CAF1ABC1CBF1ACC132
:10162000CCF1ADC1CDF1AEC1CEF1AFC1CFF1B0C102
:10163000D0F1B1C1D1F1B2C1D2F1B3C1D3F1B4C1D2
:10164000D4F1B5C1D5F1B6C1D6F1B7C1D7F1B8C1A2
:10165000D8F1B9C1D9F1B7C5B9F5B8C5BAF5B9C5A9
:10166000BBF5BAC5BCF5010155515B2756515C234A
:10167000E86A5D230E2E45EF0BF05CC157F15DC1AA
:1016800058F15B6B5C6B5D6B078E47EF0BF002C034
:10169000E0FF005001C0D8FF1000A6B24DEF0BF0E4
:1016A0000CC0A9FF0BC0A8FFA69EA69CA684F29E14
:1016B000550EA76EAA0EA76EA682F28EA694A6B2AB
:1016C0005FEF0BF00C2A1200A96EA69EA69CA680C6
:1016D000A8500C2A120004012C0E826F96EC0EF01A
:1016E0009AEC30F00C5064EC0BF0E8CF00F10C50A9
:1016F00064EC0BF0E8CF01F101AF84EF0BF00101D6
:10170000FF0E026FFF0E036F23EC30F0296790EF9E
:101710000BF00401200E826F96EC0EF095EF0BF0AB
:1017200004012D0E826F96EC0EF02DEC2EF01200BF
:1017300015941596076A0F6A106A116A126A136A7D
:10174000166A0F010D0EC16E860EC06E030EC26EBC
:101750000F01680E896E130E926E080E8A6EF30EDC
:10176000936E8B6A900E946EC80E64EC0BF0E8CF0B
:10177000E8FF1098E8A0108810A805D00E0E256E7E
:101780008E0E266E04D00F0E256E8F0E266E32EC56
:1017900031F07DEC32F0F18EF19EFC0E64EC0BF03A
:1017A000E8CF0BF00BA011800BA211820BA41184C7
:1017B0000BA81188C90E64EC0BF0E8CF1AF0CA0E22
:1017C00064EC0BF0E8CF1BF0CB0E64EC0BF0E8CF31
:1017D0001CF0CC0E64EC0BF0E8CF1DF0FB0E64ECBB
:1017E0000BF0E8CF37F0CE0E64EC0BF0E8CF14F03E
:1017F000CD0E64EC0BF0E8CF36F01F6A206A0E6A5B
:1018000001015B6B5C6B5D6B576B586BF29A01016E
:10181000476B486B496B4A6B4B6B4C6B4D6B4E6B1C
:101820004F6B506B516B526B456B466BD76AD66AE8
:101830000F01280ED56EF28A9D90B00ECD6E01017B
:101840005E6B5F6B606B616B626B636B646B656B34
:10185000666B676B686B696B536B546BCF6ACE6A50
:101860000F9A0F9C0F9E9D80760ECA6E9D8202017C
:101870003C0E006FCC6A160E64EC0BF0E8CF00F162
:10188000170E64EC0BF0E8CF01F1180E64EC0BF0CE
:10189000E8CF02F1190E64EC0BF0E8CF03F101017F
:1018A00003AF6DEF0CF09AEC30F0160E0C6E00C129
:1018B0000BF04DEC0BF0170E0C6E01C10BF04DEC64
:1018C0000BF0180E0C6E02C10BF04DEC0BF0190E64
:1018D0000C6E03C10BF04DEC0BF000C18EF101C199
:1018E0008FF102C190F103C191F100C192F101C1E8
:1018F00093F102C194F103C195F11A0E64EC0BF05F
:10190000E8CF00F11B0E64EC0BF0E8CF01F11C0EE8
:1019100064EC0BF0E8CF02F11D0E64EC0BF0E8CFA5
:1019200003F1010103AFC3EF0CF09AEC30F01A0E93
:101930000C6E00C10BF04DEC0BF01B0E0C6E01C1D8
:101940000BF04DEC0BF01C0E0C6E02C10BF04DECCD
:101950000BF01D0E0C6E03C10BF04DEC0BF01A0ECC
:1019600064EC0BF0E8CF00F11B0E64EC0BF0E8CF59
:1019700001F11C0E64EC0BF0E8CF02F11D0E64ECDB
:101980000BF0E8CF03F100C196F101C197F102C15C
:1019900098F103C199F1240EAC6E900EAB6E240E3B
:1019A000AC6E080EB86E000EB06E1F0EAF6E040166
:1019B000806B816B0F01900EAB6E0F019D8A03014E
:1019C000806B816BC26B8B92D7EC35F0D7EC35F026
:1019D000B9EC37F0B5EC33F0200E64EC0BF0E8CF47
:1019E0002FF505012F51FF0AD8A4FEEF0CF02F6B45
:1019F000200E0C6E2FC50BF04DEC0BF00501010E07
:101A0000306F3C0E316F250E64EC0BF0E8CF00F127
:101A1000260E64EC0BF0E8CF01F1270E64EC0BF01E
:101A2000E8CF02F1280E64EC0BF0E8CF03F10101DE
:101A300003AF35EF0DF09AEC30F0250E0C6E00C1BF
:101A40000BF04DEC0BF0260E0C6E01C10BF04DECC3
:101A50000BF0270E0C6E02C10BF04DEC0BF0280EB4
:101A60000C6E03C10BF04DEC0BF000C157F501C13A
:101A700058F502C159F503C15AF500C15BF501C122
:101A80005CF502C15DF503C15EF5290E64EC0BF057
:101A9000E8CF5FF5050160515F5DD8A05FC560F5D7
:101AA000210E64EC0BF0E8CF00F1220E64EC0BF099
:101AB000E8CF01F1230E64EC0BF0E8CF02F1240E25
:101AC00064EC0BF0E8CF03F1010103AF96EF0DF0EA
:101AD0009AEC30F0210E0C6E00C10BF04DEC0BF0C7
:101AE000220E0C6E01C10BF04DEC0BF0230E0C6EB0
:101AF00002C10BF04DEC0BF0240E0C6E03C10BF089
:101B00004DEC0BF0210E64EC0BF0E8CF00F1220E4F
:101B100064EC0BF0E8CF01F1230E64EC0BF0E8CF9E
:101B200002F1240E64EC0BF0E8CF03F100C161F583
:101B300001C162F502C163F503C164F5FDEC32F049
:101B4000E3EC31F03BEC31F01590C70E64EC0BF098
:101B5000E8CF00F1010100B1B1EF0DF01592B2EF45
:101B60000DF0158281AAC0EF0DF015B4BBEF0DF09A
:101B70001580C0EF0DF0F8EC37F015A05FEF38F0EE
:101B800007900001F28EF28C12AE03D012BC6EEF01
:101B900019F007B0ACEF2CF00FB0A8EF25F010BE95
:101BA000A8EF25F012B8A8EF25F000011650010AA1
:101BB000D8B4A1EF1DF081BAE6EF0DF00001165088
:101BC000040AD8B41AEF1CF0ECEF0DF00001165027
:101BD000040AD8B4DDEF1DF00301805181197F0B99
:101BE000D8B4ACEF2CF013EE00F081517F0BE1265E
:101BF000812BE7CFE8FFE00BD8B4ACEF2CF023EE5D
:101C000082F0C2513F0BD926E7CFDFFFC22BDF5056
:101C1000780AD8A4ACEF2CF0078092C100F193C1F0
:101C200001F194C102F195C103F10101040E046FA9
:101C3000000E056F000E066F000E076F85EC2FF08B
:101C400000AF2CEF0EF00101030E926F000E936FA8
:101C5000000E946F000E956F03018251720AD8B482
:101C600029EF25F08251520AD8B429EF25F082518C
:101C7000750AD8B429EF25F08251680AD8B4AAEFC2
:101C80000EF08251630AD8B466EF29F08251690AD6
:101C9000D8B4E7EF20F082517A0AD8B4FAEF21F0F5
:101CA0008251490AD8B486EF20F08251500AD8B444
:101CB000A4EF1FF08251700AD8B4E7EF1FF08251F1
:101CC000540AD8B412EF20F08251740AD8B458EFF5
:101CD00020F08251410AD8B4AFEF0FF082514B0A85
:101CE000D8B4ACEF0EF082516D0AD8B41FEF14F0E7
:101CF00082514D0AD8B438EF14F08251730AD8B427
:101D000059EF24F08251530AD8B4BEEF24F0825127
:101D10004C0AD8B4C7EF14F08251590AD8B470EF06
:101D200013F012AE01D0128C9DEF29F0040114EED5
:101D300000F080517F0BE12682C4E7FF802B120068
:101D400004010D0E826F96EC0EF00A0E826F96EC77
:101D50000EF012009BEF29F004014B0E826F96ECFF
:101D60000EF004012C0E826F96EC0EF081B802D0BA
:101D700036B630D003018351430AD8B4F1EF0EF0E8
:101D800003018351630AD8B4F3EF0EF003018351CA
:101D9000520AD8B4F5EF0EF003018351720AD8B499
:101DA000F7EF0EF003018351470AD8B4F9EF0EF0B4
:101DB00003018351670AD8B4FBEF0EF0030183518E
:101DC000540AD8B4FDEF0EF003018351740AD8B45D
:101DD0006DEF0FF003018351550AD8B4FFEF0EF0F9
:101DE00083D036807BD0369079D0368277D03692C9
:101DF00075D0368473D0369471D036866FD084C354
:101E000030F185C331F186C332F187C333F101016B
:101E1000296BE8EC30F05FEC30F000C104F101C157
:101E200005F102C106F103C107F1DBEC30F0200E31
:101E3000F86EF76AF66A0900F5CF2CF10900F5CFC4
:101E40002DF10900F5CF2EF10900F5CF2FF1090092
:101E5000F5CF30F10900F5CF31F10900F5CF32F1BE
:101E60000900F5CF33F10101296BE8EC30F05FECAC
:101E700030F085EC2FF00101006746EF0FF00167AD
:101E800046EF0FF0026746EF0FF0036701D025D051
:101E900004014E0E826F96EC0EF004016F0E826FFD
:101EA00096EC0EF004014D0E826F96EC0EF00401DC
:101EB000610E826F96EC0EF00401740E826F96EC48
:101EC0000EF00401630E826F96EC0EF00401680EB2
:101ED000826F96EC0EF09BEF29F03696CD0E0C6ECD
:101EE00036C00BF04DEC0BF0CD0E64EC0BF0E8CFF0
:101EF00036F036B006D00401630E826F96EC0EF019
:101F000005D00401430E826F96EC0EF036B206D077
:101F10000401720E826F96EC0EF005D00401520E91
:101F2000826F96EC0EF036B406D00401670E826F15
:101F300096EC0EF005D00401470E826F96EC0EF081
:101F400036B606D00401740E826F96EC0EF005D002
:101F50000401540E826F96EC0EF09BEF29F0040101
:101F6000410E826F96EC0EF003018351310AD8B412
:101F700090EF12F003018351320AD8B4C0EF11F090
:101F800003018351330AD8B449EF11F0030183519F
:101F9000340AD8B439EF10F003018351350AD8B4AC
:101FA000D9EF0FF004013F0E826F96EC0EF09BEF1D
:101FB00029F003018451300AD8B4FFEF0FF0030178
:101FC0008451310AD8B402EF10F003018451650A3C
:101FD000D8B4F3EF0FF003018451640AD8B4F6EFDC
:101FE0000FF003EF10F03790F7EF0FF03780FB0E94
:101FF0000C6E37C00BF04DEC0BF003EF10F08B9034
:1020000003EF10F08B800401350E826F96EC0EF01A
:1020100004012C0E826F96EC0EF08BB017EF10F0CF
:102020000401300E826F96EC0EF01CEF10F00401EC
:10203000310E826F96EC0EF004012C0E826F96EC3E
:102040000EF0FB0E64EC0BF0E8CF37F037A030EF6A
:1020500010F00401640E826F96EC0EF035EF10F074
:102060000401650E826F96EC0EF037EF10F09BEFD7
:1020700029F0CC0E64EC0BF0E8CF0BF004012C0E31
:10208000826F96EC0EF003018451310AD8B45DEFF3
:1020900010F003018451300AD8B45FEF10F003014F
:1020A00084514D0AD8B469EF10F003018451540AE9
:1020B000D8B470EF10F087EF10F08A8401D08A94C2
:1020C0000BAE04D00BAC02D00BBA21D0E00E0B1239
:1020D00018D01F0E0B168539E844E00B0B1211D0F7
:1020E000E00E0B16DBEC30F085C332F186C333F122
:1020F0000101296BE8EC30F05FEC30F000511F0B70
:102100000B12CC0E0C6E0BC00BF04DEC0BF004015F
:10211000340E826F96EC0EF004012C0E826F96EC5A
:102120000EF0CC0E64EC0BF0E8CF1DF08AB406D0B4
:102130000401300E826F96EC0EF005D00401310ED2
:10214000826F96EC0EF004012C0E826F96EC0EF06E
:102150001D38E840070BE8CF82F40401300E8227D7
:1021600096EC0EF004012C0E826F96EC0EF09AECB9
:1021700030F01D501F0BE8CF00F123EC30F032C1DE
:1021800082F40401300E822796EC0EF033C182F403
:102190000401300E822796EC0EF004012C0E826FA3
:1021A00096EC0EF09AEC30F030C000F100AF0BD09E
:1021B000FF0E016FFF0E026FFF0E036F04012D0E65
:1021C000826F96EC0EF023EC30F031C182F4040102
:1021D000300E822796EC0EF032C182F40401300EEC
:1021E000822796EC0EF033C182F40401300E822770
:1021F00096EC0EF004012C0E826F96EC0EF09AEC29
:1022000030F02FC000F123EC30F031C182F4040132
:10221000300E822796EC0EF032C182F40401300EAB
:10222000822796EC0EF033C182F40401300E82272F
:1022300096EC0EF004012C0E826F96EC0EF09AECE8
:1022400030F031C000F100AF0BD0FF0E016FFF0E78
:10225000026FFF0E036F04012D0E826F96EC0EF0DD
:1022600023EC30F031C182F40401300E822796EC69
:102270000EF032C182F40401300E822796EC0EF08B
:1022800033C182F40401300E822796EC0EF09BEFEE
:1022900029F0CB0E64EC0BF0E8CF0BF004012C0E10
:1022A000826F96EC0EF003018451450AD8B46DEFAD
:1022B00011F003018451440AD8B470EF11F0030106
:1022C0008451300AD8B473EF11F003018451310AFC
:1022D000D8B477EF11F082EF11F00B9E7CEF11F084
:1022E0000B8E7CEF11F0FC0E0B167CEF11F0FC0E48
:1022F0000B160B807CEF11F0CB0E0C6E0BC00BF0AD
:102300004DEC0BF00401330E826F96EC0EF00401DD
:102310002C0E826F96EC0EF0CB0E64EC0BF0E8CF37
:102320001CF01CBE9BEF11F00401450E826F96EC71
:102330000EF0A0EF11F00401440E826F96EC0EF047
:1023400004012C0E826F96EC0EF00401300E826FA9
:1023500096EC0EF004012C0E826F96EC0EF01CB081
:10236000B9EF11F00401300E826F96EC0EF0BEEF63
:1023700011F00401310E826F96EC0EF09BEF29F004
:10238000CA0E64EC0BF0E8CF0BF004012C0E826F48
:1023900096EC0EF003018451450AD8B4FCEF11F01D
:1023A00003018451440AD8B4FFEF11F003018451B2
:1023B0004D0AD8B408EF12F003018451410AD8B491
:1023C00002EF12F003018451460AD8B405EF12F06F
:1023D00003018451560AD8B410EF12F0030184515E
:1023E000500AD8B41BEF12F003018451520AD8B43A
:1023F0001EEF12F027EF12F00B9E21EF12F00B8E62
:1024000021EF12F00B9C21EF12F00B8C21EF12F058
:10241000FC0E0B1685C3E8FF030B0B1221EF12F025
:10242000C70E0B1685C3E8FF070BE846E846E846EB
:102430000B1221EF12F00B8421EF12F00B9421EF1D
:1024400012F0CA0E0C6E0BC00BF04DEC0BF0CA0E66
:1024500064EC0BF0E8CF1BF00401320E826F96ECB7
:102460000EF004012C0E826F96EC0EF01BBE40EFB6
:1024700012F00401450E826F96EC0EF045EF12F05B
:102480000401440E826F96EC0EF004012C0E826F54
:1024900096EC0EF01BC0E8FF030BE8CF82F40401BA
:1024A000300E822796EC0EF004012C0E826F96EC13
:1024B0000EF01BBC63EF12F00401410E826F96EC2C
:1024C0000EF068EF12F00401460E826F96EC0EF0EB
:1024D00004012C0E826F96EC0EF01BC0E8FF380B47
:1024E000E842E842E842E8CF82F40401300E822755
:1024F00096EC0EF004012C0E826F96EC0EF01BB4DD
:1025000089EF12F00401520E826F96EC0EF08EEFFE
:1025100012F00401500E826F96EC0EF09BEF29F042
:10252000C90E64EC0BF0E8CF0BF004012C0E826FA7
:1025300096EC0EF003018451450AD8B4AEEF12F0C8
:1025400003018451440AD8B4B1EF12F0030184515D
:102550004D0AD8B4B4EF12F0C2EF12F00B9EBCEFEC
:1025600012F00B8EBCEF12F0F80E0B1685C3E8FFCD
:10257000070B0B12BCEF12F0C90E0C6E0BC00BF068
:102580004DEC0BF00401310E826F96EC0EF004015D
:102590002C0E826F96EC0EF0C90E64EC0BF0E8CFB7
:1025A0001AF01ABE06D00401450E826F96EC0EF0AA
:1025B00005D00401440E826F96EC0EF004012C0E3F
:1025C000826F96EC0EF01AC0E8FF070BE8CF82F49A
:1025D0000401300E822796EC0EF004012C0E826F5F
:1025E00096EC0EF007809AEC30F02BC0E8FF003B31
:1025F00000430043030B23EC30F033C182F40401A9
:10260000300E822796EC0EF004012C0E826F96ECB1
:102610000EF09AEC30F02BC001F1019F019D2CC00F
:1026200000F1010123EC30F02FC182F40401300EDF
:10263000822796EC0EF030C182F40401300E82271E
:1026400096EC0EF031C182F40401300E822796EC34
:102650000EF032C182F40401300E822796EC0EF0A7
:1026600033C182F40401300E822796EC0EF004018F
:102670002C0E826F96EC0EF09AEC30F02DC001F12A
:102680002EC000F1D89001330033D89001330033CD
:10269000010123EC30F02FC182F40401300E8227B7
:1026A00096EC0EF030C182F40401300E822796ECD5
:1026B0000EF031C182F40401300E822796EC0EF048
:1026C00032C182F40401300E822796EC0EF033C141
:1026D00082F40401300E822796EC0EF09BEF29F075
:1026E000FC0E64EC0BF0E8CF0BF003018351520AAF
:1026F000D8B4A7EF13F003018351720AD8B4AAEF3C
:1027000013F003018351500AD8B4ADEF13F0030165
:102710008351700AD8B4B0EF13F003018351550A06
:10272000D8B4B3EF13F003018351750AD8B4B6EFF0
:1027300013F003018351430AD8B4BFEF13F0030130
:102740008351630AD8B4C2EF13F0CBEF13F00B90B0
:10275000C5EF13F00B80C5EF13F00B92C5EF13F02C
:102760000B82C5EF13F00B94C5EF13F00B84C5EF8C
:1027700013F00B96C5EF13F00B86C5EF13F00B9813
:10278000C5EF13F00B88C5EF13F0FC0E0C6E0BC0F9
:102790000BF04DEC0BF00401590E826F96EC0EF02D
:1027A0001190119211941198FC0E64EC0BF0E8CF8B
:1027B0000BF00BA011800BA211820BA411840BA8AB
:1027C000118811A0EBEF13F00401520E826F96EC0A
:1027D0000EF0F0EF13F00401720E826F96EC0EF023
:1027E00011A8FAEF13F00401430E826F96EC0EF07D
:1027F000FFEF13F00401630E826F96EC0EF011A24E
:1028000009EF14F00401500E826F96EC0EF00EEFFB
:1028100014F00401700E826F96EC0EF011A418EF04
:1028200014F00401550E826F96EC0EF01DEF14F0BB
:102830000401750E826F96EC0EF09BEF29F00401F7
:102840006D0E826F96EC0EF003018351300AD8B4FE
:1028500077EF14F003018351310AD8B48AEF14F0F2
:1028600003018351320AD8B49DEF14F09DEF29F093
:1028700004014D0E826F96EC0EF0DBEC30F084C359
:1028800031F185C332F186C333F10101296BE8ECE4
:1028900030F05FEC30F003018351300AD8B45FEFC1
:1028A00014F003018351310AD8B467EF14F0030127
:1028B0008351320AD8B46FEF14F09DEF29F0FD0E6A
:1028C0000C6E00C10BF04DEC0BF077EF14F0FE0E28
:1028D0000C6E00C10BF04DEC0BF08AEF14F0FF0E04
:1028E0000C6E00C10BF04DEC0BF09DEF14F00401E9
:1028F000300E826F96EC0EF004012C0E826F96EC77
:102900000EF09AEC30F0FD0E64EC0BF0E8CF00F125
:10291000AEEF14F00401310E826F96EC0EF004015C
:102920002C0E826F96EC0EF09AEC30F0FE0E64ECFA
:102930000BF0E8CF00F1AEEF14F00401320E826F1D
:1029400096EC0EF09AEC30F004012C0E826F96ECAF
:102950000EF0FF0E64EC0BF0E8CF00F123EC30F04A
:1029600031C182F40401300E822796EC0EF032C1A0
:1029700082F40401300E822796EC0EF033C182F40B
:102980000401300E822796EC0EF09BEF29F0030134
:102990008351300AD8B41BEF1AF003018351310A76
:1029A000D8B448EF1BF003018351320AD8B4B6EF14
:1029B0001BF003018351330AD8B4C6EF1BF00301A7
:1029C0008351340AD8B421EF1CF003018351350A36
:1029D000D8B4F5EF1DF003018351360AD8B423EFC4
:1029E0001EF003018351370AD8B4F3EF17F0030147
:1029F0008351380AD8B491EF18F003018351440A87
:102A0000D8B41FEF16F003018351640AD8B43FEF26
:102A100016F003018351460AD8B4FAEF1CF0030103
:102A200083514D0AD8B46CEF16F0030183516D0A3F
:102A3000D8B486EF16F0030183515A0AD8B4C2EF16
:102A40001AF003018351490AD8B423EF1FF00301A0
:102A50008351500AD8B455EF1EF003018351540A34
:102A6000D8B4CEEF1EF003018351630AD8B4A6EFA9
:102A700016F003018351430AD8B49EEF17F0030107
:102A80008351730AD8B4A4EF16F003018351610A8D
:102A9000D8B46CEF15F003018351650AD8B46BEF1D
:102AA0001AF003018351450AD8B479EF1AF00301F3
:102AB0008351620AD8B487EF1AF003018351420AA6
:102AC000D8B495EF1AF003018351760AD8B4A3EF76
:102AD0001AF0D8A49DEF29F004014C0E826F96ECF9
:102AE0000EF00401610E826F96EC0EF0E3EC31F013
:102AF00004012C0E826F96EC0EF09AEC30F0AFC50C
:102B000000F1010123EC30F031C182F40401300EF8
:102B1000822796EC0EF032C182F40401300E822737
:102B200096EC0EF033C182F40401300E822796EC4D
:102B30000EF004012C0E826F96EC0EF09AEC30F041
:102B4000B0C500F1010123EC30F031C182F4040181
:102B5000300E822796EC0EF032C182F40401300E62
:102B6000822796EC0EF033C182F40401300E8227E6
:102B700096EC0EF004012C0E826F96EC0EF09AEC9F
:102B800030F0B1C500F1010123EC30F031C182F425
:102B90000401300E822796EC0EF032C182F404015B
:102BA000300E822796EC0EF033C182F40401300E11
:102BB000822796EC0EF004012C0E826F96EC0EF03C
:102BC0009AEC30F0B2C500F1010123EC30F031C1D4
:102BD00082F40401300E822796EC0EF032C182F4AA
:102BE0000401300E822796EC0EF033C182F404010A
:102BF000300E822796EC0EF004012C0E826F96ECBC
:102C00000EF09AEC30F0B6C500F1010123EC30F083
:102C100031C182F40401300E822796EC0EF032C1ED
:102C200082F40401300E822796EC0EF033C182F458
:102C30000401300E822796EC0EF051EF1EF00301D6
:102C40008451300AD8B42BEF16F003018451310AB5
:102C5000D8B42FEF16F01592159630EF16F01582B6
:102C6000C70E64EC0BF0E8CF00F10101008115A262
:102C70000091C70E0C6E00C10BF04DEC0BF0C70EAF
:102C800064EC0BF0E8CF00F1010100B14BEF16F05E
:102C900015924CEF16F0158204014C0E826F96ECE3
:102CA0000EF00401640E826F96EC0EF004012C0EFF
:102CB000826F96EC0EF015B265EF16F00401300E3F
:102CC000826F96EC0EF06AEF16F00401310E826FFF
:102CD00096EC0EF09BEF29F0DBEC30F084C333F17F
:102CE000E8EC30F05FEC30F0200E0C6E00C10BF021
:102CF0004DEC0BF000C12FF505012F51000A06E045
:102D000005012F51010A02E07DEC32F004014C0E66
:102D1000826F96EC0EF004014D0E826F96EC0EF071
:102D200004012C0E826F96EC0EF09AEC30F02FC559
:102D300000F123EC30F033C182F40401300E82271D
:102D400096EC0EF051EF1EF05FEF38F004014C0EE0
:102D5000826F96EC0EF00401630E826F96EC0EF01B
:102D60003BEC31F004012C0E826F96EC0EF0BBECC4
:102D700016F051EF1EF09AEC30F0B5C500F10101EC
:102D8000003B0F0E001723EC30F033C182F4040136
:102D9000300E822796EC0EF0B5C500F101010F0E42
:102DA0000101001723EC30F033C182F40401300E2E
:102DB000822796EC0EF004012D0E826F96EC0EF039
:102DC000B4C500F10101003B0F0E001723EC30F0F9
:102DD00033C182F40401300E822796EC0EF0B4C5A4
:102DE00000F101010F0E0101001723EC30F033C197
:102DF00082F40401300E822796EC0EF004012D0EB1
:102E0000826F96EC0EF0B3C500F10101003B0F0E8E
:102E1000001723EC30F033C182F40401300E822716
:102E200096EC0EF0B3C500F101010F0E0101001781
:102E300023EC30F033C182F40401300E822796EC8B
:102E40000EF00401200E826F96EC0EF0B2C500F178
:102E50000F0E0101001723EC30F033C182F404019E
:102E6000300E822796EC0EF00401200E826F96EC55
:102E70000EF0B1C500F101010101003B0F0E00177A
:102E800023EC30F033C182F40401300E822796EC3B
:102E90000EF0B1C500F101010F0E0101001723EC86
:102EA00030F033C182F40401300E822796EC0EF02C
:102EB00004013A0E826F96EC0EF0B0C500F10101EC
:102EC000003B0F0E001723EC30F033C182F40401F5
:102ED000300E822796EC0EF0B0C500F101010F0E06
:102EE0000101001723EC30F033C182F40401300EED
:102EF000822796EC0EF004013A0E826F96EC0EF0EB
:102F0000AFC500F10101003B0F0E001723EC30F0BC
:102F100033C182F40401300E822796EC0EF0AFC567
:102F200000F101010F0E001723EC30F033C182F4E1
:102F30000401300E822796EC0EF0120084C3E8FFE5
:102F40000F0BE83AE8CFB5F585C3E8FF0F0B050195
:102F5000B51387C3E8FF0F0BE83AE8CFB4F588C391
:102F6000E8FF0F0B0501B4138AC3E8FF0F0BE83A23
:102F7000E8CFB3F58BC3E8FF0F0B0501B3138DC387
:102F8000E8FF0F0BE8CFB2F58FC3E8FF0F0BE83A6D
:102F9000E8CFB1F590C3E8FF0F0B0501B11392C361
:102FA000E8FF0F0BE83AE8CFB0F593C3E8FF0F0B4B
:102FB0000501B01395C3E8FF0F0BE83AE8CFAFF572
:102FC00096C3E8FF0F0B0501AF1396EC31F0040137
:102FD0004C0E826F96EC0EF00401430E826F96EC5D
:102FE0000EF0B0EF16F0078404014C0E826F96ECE1
:102FF0000EF00401370E826F96EC0EF004012C0ED9
:10300000826F96EC0EF005012E51130A06E00501C1
:103010002E51170A0DE08EEF18F00101000E006F1F
:10302000000E016F100E026F000E036F21EF18F0FB
:103030000101000E006F000E016F000E026F010E05
:10304000036F23EC30F02AC182F40401300E822792
:1030500096EC0EF02BC182F40401300E822796EC20
:103060000EF02CC182F40401300E822796EC0EF093
:103070002DC182F40401300E822796EC0EF02EC191
:1030800082F40401300E822796EC0EF02FC182F4F8
:103090000401300E822796EC0EF030C182F4040158
:1030A000300E822796EC0EF031C182F40401300E0E
:1030B000822796EC0EF032C182F40401300E822792
:1030C00096EC0EF033C182F40401300E822796ECA8
:1030D0000EF004012C0E826F96EC0EF00101100E22
:1030E000006F000E016F000E026F000E036F23ECE5
:1030F00030F031C182F40401300E822796EC0EF0DC
:1031000032C182F40401300E822796EC0EF033C1F6
:1031100082F40401300E822796EC0EF0079451EFF2
:103120001EF00501216B226B236B246B04014C0EF6
:10313000826F96EC0EF00401380E826F96EC0EF062
:1031400004012C0E826F96EC0EF00101100E006F40
:10315000000E016F000E026F000E036F23EC30F0C3
:103160002AC182F40401300E822796EC0EF02BC1A6
:1031700082F40401300E822796EC0EF02CC182F40A
:103180000401300E822796EC0EF02DC182F404016A
:10319000300E822796EC0EF02EC182F40401300E20
:1031A000822796EC0EF02FC182F40401300E8227A4
:1031B00096EC0EF030C182F40401300E822796ECBA
:1031C0000EF031C182F40401300E822796EC0EF02D
:1031D00032C182F40401300E822796EC0EF033C126
:1031E00082F40401300E822796EC0EF004012C0EBE
:1031F000826F96EC0EF025C500F126C501F127C5BA
:1032000002F128C503F10101100E046F000E056FD5
:10321000000E066F000E076FB6EC2FF000C133F5FD
:1032200001C134F502C135F503C136F523EC30F0A8
:103230002AC182F40401300E822796EC0EF02BC1D5
:1032400082F40401300E822796EC0EF02CC182F439
:103250000401300E822796EC0EF02DC182F4040199
:10326000300E822796EC0EF02EC182F40401300E4F
:10327000822796EC0EF02FC182F40401300E8227D3
:1032800096EC0EF030C182F40401300E822796ECE9
:103290000EF031C182F40401300E822796EC0EF05C
:1032A00032C182F40401300E822796EC0EF033C155
:1032B00082F40401300E822796EC0EF0A0EC0EF0A2
:1032C000050133676BEF19F034676BEF19F0356761
:1032D0006BEF19F0366702D00AEF1AF0129E129CBB
:1032E00021C500F122C501F123C502F124C503F176
:1032F000899A400EC76E200EC66E9E96C69E0B0E15
:10330000C96EFF0E9EB602D0E82EFCD79E96C69ED2
:1033100002C1C9FFFF0E9EB602D0E82EFCD79E96D2
:10332000C69E01C1C9FFFF0E9EB602D0E82EFCD793
:103330009E96C69E00C1C9FFFF0E9EB602D0E82E23
:10334000FCD79E96C69EC952FF0E9EB602D0E82EAE
:10335000FCD70501100E326F040114EE00F080510D
:103360007F0BE1269E96C69EC952FF0E9EB602D0E6
:10337000E82EFCD7C9CFE7FF0401802B0501322FCF
:10338000ACEF19F0898A33C500F134C501F135C5B8
:1033900002F136C503F10101010E046F000E056F45
:1033A000000E066F000E076F85EC2FF000C133F59D
:1033B00001C134F502C135F503C136F505013367A6
:1033C000E9EF19F03467E9EF19F03567E9EF19F023
:1033D000366702D00AEF1AF021C500F122C501F1CB
:1033E00023C502F124C503F10101100E046F000E84
:1033F000056F000E066F000E076F8AEC2FF000C1FC
:1034000021F501C122F502C123F503C124F5128E75
:103410009DEF29F00401450E826F96EC0EF0040139
:103420004F0E826F96EC0EF00401460E826F96EC02
:103430000EF051EF1EF00784B9EC37F09AEC30F043
:103440002DC500F123EC30F004014C0E826F96EC98
:103450000EF00401300E826F96EC0EF004012C0E7B
:10346000826F96EC0EF031C182F40401300E822797
:1034700096EC0EF032C182F40401300E822796ECF5
:103480000EF033C182F40401300E822796EC0EF068
:1034900004012C0E826F96EC0EF09AEC30F02EC5E3
:1034A00000F123EC30F031C182F40401300E8227A8
:1034B00096EC0EF032C182F40401300E822796ECB5
:1034C0000EF033C182F40401300E822796EC0EF028
:1034D000079451EF1EF004014C0E826F96EC0EF033
:1034E0000401650E826F96EC0EF059EC33F051EF4B
:1034F0001EF004014C0E826F96EC0EF00401450E96
:10350000826F96EC0EF070EC33F051EF1EF0040178
:103510004C0E826F96EC0EF00401620E826F96ECF8
:103520000EF09EEC33F051EF1EF004014C0E826F52
:1035300096EC0EF00401420E826F96EC0EF087ECD2
:1035400033F051EF1EF004014C0E826F96EC0EF03A
:103550000401760E826F96EC0EF004012C0E826F41
:1035600096EC0EF010A807D00401310E826F96EC95
:103570000EF051EF1EF00401300E826F96EC0EF04B
:1035800051EF1EF004014C0E826F96EC0EF0040118
:103590005A0E826F96EC0EF004012C0E826F96ECA0
:1035A0000EF0B9EC37F09AEC30F005012E51130A09
:1035B00006E005012E51170A0DE0F3EF1AF00101A4
:1035C000000E006F000E016F100E026F000E036FF1
:1035D000F3EF1AF00101000E006F000E016F000EF4
:1035E000026F010E036F0101100E046F000E056FD4
:1035F000000E066F000E076FB6EC2FF023EC30F0D4
:103600002AC182F40401300E822796EC0EF02BC101
:1036100082F40401300E822796EC0EF02CC182F465
:103620000401300E822796EC0EF02DC182F40401C5
:10363000300E822796EC0EF02EC182F40401300E7B
:10364000822796EC0EF02FC182F40401300E8227FF
:1036500096EC0EF030C182F40401300E822796EC15
:103660000EF031C182F40401300E822796EC0EF088
:1036700032C182F40401300E822796EC0EF033C181
:1036800082F40401300E822796EC0EF051EF1EF00A
:10369000078404014C0E826F96EC0EF00401310E8B
:1036A000826F96EC0EF004012C0E826F96EC0EF0F9
:1036B00025C500F126C501F127C502F128C503F192
:1036C0000101100E046F000E056F000E066F000E54
:1036D000076FB6EC2FF023EC30F02AC182F404011E
:1036E000300E822796EC0EF02BC182F40401300ECE
:1036F000822796EC0EF02CC182F40401300E822752
:1037000096EC0EF02DC182F40401300E822796EC67
:103710000EF02EC182F40401300E822796EC0EF0DA
:103720002FC182F40401300E822796EC0EF030C1D6
:1037300082F40401300E822796EC0EF031C182F43F
:103740000401300E822796EC0EF032C182F404019F
:10375000300E822796EC0EF033C182F40401300E55
:10376000822796EC0EF0079451EF1EF007840401B7
:103770004C0E826F96EC0EF00401320E826F96ECC6
:103780000EF08DEC35F0079451EF1EF0078437B042
:10379000CCEF1BF0DFEF1BF0010E166E04014C0E98
:1037A000826F96EC0EF00401330E826F96EC0EF0F1
:1037B000EAEC35F0000E166E079453EF1BF0020E84
:1037C000166EEAEC35F08B800501010E306F3C0E71
:1037D000316F01015E6B5F6B606B616B626B636B82
:1037E000646B656B666B676B686B696B536B546B73
:1037F000CF6ACE6A0F9A0F9C0F9E030E166E0401BD
:103800004C0E826F96EC0EF00401330E826F96EC34
:103810000EF004012C0E826F96EC0EF004012D0EBA
:10382000826F96EC0EF00401310E826F96EC0EF072
:103830009BEF29F0EAEC35F0000E166E8B909DEFB1
:1038400029F0078404014C0E826F96EC0EF00401FF
:10385000340E826F96EC0EF004012C0E826F96EC03
:103860000EF0DBEC30F084C32AF185C32BF186C364
:103870002CF187C32DF188C32EF189C32FF18AC3A0
:1038800030F18BC331F18CC332F18DC333F10101BF
:10389000296BE8EC30F05FEC30F0100E046F000E96
:1038A000056F000E066F000E076F96EC2FF000C13B
:1038B00021F501C122F502C123F503C124F56CEC09
:1038C00037F038C5AFF539C5B0F53AC5B1F53BC5E8
:1038D000B2F53CC5B3F53DC5B4F53EC5B5F5BBEC99
:1038E00016F004012C0E826F96EC0EF03FC500F12D
:1038F00040C501F141C502F142C503F10101000ECD
:10390000046F000E056F010E066F000E076FB6EC18
:103910002FF023EC30F0296790EF1CF095EF1CF0AE
:1039200004012D0E826F96EC0EF030C182F404017A
:10393000300E822796EC0EF031C182F40401300E75
:10394000822796EC0EF004012E0E826F96EC0EF09C
:1039500032C182F40401300E822796EC0EF033C19E
:1039600082F40401300E822796EC0EF004012C0E36
:10397000826F96EC0EF09AEC30F043C500F144C52E
:1039800001F1C7EC2AF004012C0E826F96EC0EF0C8
:103990009AEC30F045C500F123EC30F031C182F4EF
:1039A0000401300E822796EC0EF032C182F404013D
:1039B000300E822796EC0EF033C182F40401300EF3
:1039C000822796EC0EF004012C0E826F96EC0EF01E
:1039D00037C5E8FFE8B806D00401300E826F96ECD8
:1039E0000EF005D00401310E826F96EC0EF00794B4
:1039F00051EF1EF0DBEC30F085C32AF186C32BF1CA
:103A000087C32CF188C32DF189C32EF18AC32FF10E
:103A10008BC330F18CC331F18DC332F18EC333F1DE
:103A20000101296BE8EC30F05FEC30F00101010E90
:103A3000046F000E056F000E066F000E076F85EC19
:103A40002FF0100E046F000E056F000E066F000EB3
:103A5000076F96EC2FF000C129F501C12AF502C1CC
:103A60002BF503C12CF514EC35F004014C0E826FDC
:103A700096EC0EF00401460E826F96EC0EF00401F7
:103A80002C0E826F96EC0EF025C500F126C501F1D3
:103A900027C502F128C503F10101100E046F000EC5
:103AA000056F000E066F000E076FB6EC2FF023ECCB
:103AB00030F02AC182F40401300E822796EC0EF019
:103AC0002BC182F40401300E822796EC0EF02CC13B
:103AD00082F40401300E822796EC0EF02DC182F4A0
:103AE0000401300E822796EC0EF02EC182F4040100
:103AF000300E822796EC0EF02FC182F40401300EB6
:103B0000822796EC0EF030C182F40401300E822739
:103B100096EC0EF031C182F40401300E822796EC4F
:103B20000EF032C182F40401300E822796EC0EF0C2
:103B300033C182F40401300E822796EC0EF051EF6F
:103B40001EF037B0A6EF1DF0020E166EEAEC35F04F
:103B500000011650020AD8B4C4EF1DF005012F5120
:103B6000010AD8B4BAEF1DF015B2BFEF1DF081BA4B
:103B7000BFEF1DF0000E166E15849DEF29F0050EA7
:103B8000166E15845FEF38F08B8001015E6B5F6B02
:103B9000606B616B626B636B646B656B666B676BB1
:103BA000686B696B536B546BCF6ACE6A0F9A0F9C2C
:103BB0000F9E030E166E9DEF29F0EAEC35F005011D
:103BC0002F51010AD8B4EBEF1DF015B2F0EF1DF044
:103BD00081BAF0EF1DF0000E166E15849DEF29F0EE
:103BE000050E166E15845FEF38F004014C0E826FDF
:103BF00096EC0EF00401350E826F96EC0EF0040187
:103C00002C0E826F96EC0EF09AEC30F00784B9C55A
:103C100000F1079423EC30F031C182F40401300E3E
:103C2000822796EC0EF032C182F40401300E822716
:103C300096EC0EF033C182F40401300E822796EC2C
:103C40000EF051EF1EF0ADEC35F09AEC30F037C5C8
:103C500000F123EC30F004014C0E826F96EC0EF074
:103C60000401360E826F96EC0EF004012C0E826F6A
:103C700096EC0EF031C182F40401300E822796ECEE
:103C80000EF032C182F40401300E822796EC0EF061
:103C900033C182F40401300E822796EC0EF051EF0E
:103CA0001EF0A0EC0EF09DEF29F004014C0E826F87
:103CB00096EC0EF00401500E826F96EC0EF00401AB
:103CC0002C0E826F96EC0EF085C32AF186C32BF181
:103CD00087C32CF188C32DF189C32EF18AC32FF13C
:103CE0008BC330F18CC331F18DC332F18EC333F10C
:103CF0000101E8EC30F05FEC30F003018451530A2D
:103D00000DE0030184514D0A38E00401780E826F02
:103D100096EC0EF0A0EC0EF09DEF29F00401530E8E
:103D2000826F96EC0EF0250E0C6E00C10BF04DEC80
:103D30000BF0260E0C6E01C10BF04DEC0BF0270EB4
:103D40000C6E02C10BF04DEC0BF0280E0C6E03C193
:103D50000BF04DEC0BF000C157F501C158F502C155
:103D600059F503C15AF500C15BF501C15CF502C10B
:103D70005DF503C15EF532EF1FF004014D0E826F59
:103D800096EC0EF0290E0C6E00C10BF04DEC0BF012
:103D900000C15FF500C160F532EF1FF004014C0E69
:103DA000826F96EC0EF00401540E826F96EC0EF0CA
:103DB00004012C0E826F96EC0EF084C32AF185C3A9
:103DC0002BF186C32CF187C32DF188C32EF189C353
:103DD0002FF18AC330F18BC331F18DC332F18EC321
:103DE00033F10101E8EC30F05FEC30F00101000E3E
:103DF000046F000E056F010E066F000E076F96EC44
:103E00002FF0210E0C6E00C10BF04DEC0BF0220ECA
:103E10000C6E01C10BF04DEC0BF0230E0C6E02C1C9
:103E20000BF04DEC0BF0240E0C6E03C10BF04DECBF
:103E30000BF000C161F501C162F502C163F503C178
:103E400064F532EF1FF004014C0E826F96EC0EF019
:103E50000401490E826F96EC0EF004012C0E826F65
:103E600096EC0EF0250E64EC0BF0E8CF00F1260E78
:103E700064EC0BF0E8CF01F1270E64EC0BF0E8CF17
:103E800002F1280E64EC0BF0E8CF03F123EC30F0E4
:103E9000E6EC2DF00401730E826F96EC0EF0040137
:103EA0002C0E826F96EC0EF09AEC30F0290E64EC3A
:103EB0000BF0E8CF00F123EC30F0E6EC2DF004013C
:103EC0006D0E826F96EC0EF004012C0E826F96EC54
:103ED0000EF05BC500F15CC501F15DC502F15EC588
:103EE00003F123EC30F0E6EC2DF00401730E826F49
:103EF00096EC0EF004012C0E826F96EC0EF09AEC0C
:103F000030F060C500F123EC30F0E6EC2DF0040158
:103F10006D0E826F96EC0EF004012C0E826F96EC03
:103F20000EF061C500F162C501F163C502F164C51F
:103F300003F1B8EC29F004012C0E826F96EC0EF020
:103F4000A0EC0EF09DEF29F083C32AF184C32BF17E
:103F500085C32CF186C32DF187C32EF188C32FF1C1
:103F600089C330F18AC331F18BC332F18CC333F191
:103F70000101E8EC30F05FEC30F0160E0C6E00C181
:103F80000BF04DEC0BF0170E0C6E01C10BF04DEC6D
:103F90000BF0180E0C6E02C10BF04DEC0BF0190E6D
:103FA0000C6E03C10BF04DEC0BF000C18EF101C1A2
:103FB0008FF102C190F103C191F100C192F101C1F1
:103FC00093F102C194F103C195F186EF20F083C310
:103FD0002AF184C32BF185C32CF186C32DF187C34D
:103FE0002EF188C32FF189C330F18AC331F18BC31D
:103FF00032F18CC333F10101E8EC30F05FEC30F0CA
:1040000000C18EF101C18FF102C190F103C191F1A4
:1040100000C192F101C193F102C194F103C195F184
:1040200086EF20F083C32AF184C32BF185C32CF1E2
:1040300086C32DF187C32EF188C32FF189C330F1D8
:104040008AC331F18CC332F18DC333F10101E8EC45
:1040500030F05FEC30F00101000E046F000E056FD0
:10406000010E066F000E076F96EC2FF01A0E0C6E05
:1040700000C10BF04DEC0BF01B0E0C6E01C10BF0F0
:104080004DEC0BF01C0E0C6E02C10BF04DEC0BF066
:104090001D0E0C6E03C10BF04DEC0BF000C196F140
:1040A00001C197F102C198F103C199F186EF20F0A7
:1040B00083C32AF184C32BF185C32CF186C32DF170
:1040C00087C32EF188C32FF189C330F18AC331F140
:1040D0008CC332F18DC333F10101E8EC30F05FECB9
:1040E00030F00101000E046F000E056F010E066F27
:1040F000000E076F96EC2FF000C196F101C197F109
:1041000002C198F103C199F186EF20F0160E64EC1C
:104110000BF0E8CF00F1170E64EC0BF0E8CF01F1E3
:10412000180E64EC0BF0E8CF02F1190E64EC0BF002
:10413000E8CF03F123EC30F0E6EC2DF00401730E30
:10414000826F96EC0EF004012C0E826F96EC0EF04E
:104150008EC100F18FC101F190C102F191C103F153
:1041600023EC30F0E6EC2DF00401730E826F96EC38
:104170000EF004012C0E826F96EC0EF01A0E64EC19
:104180000BF0E8CF00F11B0E64EC0BF0E8CF01F16F
:104190001C0E64EC0BF0E8CF02F11D0E64EC0BF08A
:1041A000E8CF03F1B8EC29F004012C0E826F96ECF5
:1041B0000EF096C100F197C101F198C102F199C1C9
:1041C00003F1B8EC29F0A0EC0EF09DEF29F004010A
:1041D000690E826F96EC0EF004012C0E826F96EC45
:1041E0000EF00101040E006F000E016F000E026F51
:1041F000000E036F23EC30F02CC182F40401300E6A
:10420000822796EC0EF02DC182F40401300E822735
:1042100096EC0EF02EC182F40401300E822796EC4B
:104220000EF02FC182F40401300E822796EC0EF0BE
:1042300030C182F40401300E822796EC0EF031C1B9
:1042400082F40401300E822796EC0EF032C182F423
:104250000401300E822796EC0EF033C182F4040183
:10426000300E822796EC0EF004012C0E826F96EC35
:104270000EF00101060E006F000E016F000E026FBE
:10428000000E036F23EC30F02CC182F40401300ED9
:10429000822796EC0EF02DC182F40401300E8227A5
:1042A00096EC0EF02EC182F40401300E822796ECBB
:1042B0000EF02FC182F40401300E822796EC0EF02E
:1042C00030C182F40401300E822796EC0EF031C129
:1042D00082F40401300E822796EC0EF032C182F493
:1042E0000401300E822796EC0EF033C182F40401F3
:1042F000300E822796EC0EF004012C0E826F96ECA5
:104300000EF00101490E006F000E016F000E026FEA
:10431000000E036F23EC30F02CC182F40401300E48
:10432000822796EC0EF02DC182F40401300E822714
:1043300096EC0EF02EC182F40401300E822796EC2A
:104340000EF02FC182F40401300E822796EC0EF09D
:1043500030C182F40401300E822796EC0EF031C198
:1043600082F40401300E822796EC0EF032C182F402
:104370000401300E822796EC0EF033C182F4040162
:10438000300E822796EC0EF004012C0E826F96EC14
:104390000EF0200EF86EF76AF66A04010900F5CFF8
:1043A00082F496EC0EF00900F5CF82F496EC0EF054
:1043B0000900F5CF82F496EC0EF00900F5CF82F4F7
:1043C00096EC0EF00900F5CF82F496EC0EF00900A1
:1043D000F5CF82F496EC0EF00900F5CF82F496EC5E
:1043E0000EF00900F5CF82F496EC0EF0A0EC0EF082
:1043F0009DEF29F08351630AD8A49BEF29F08451E3
:10440000610AD8A49BEF29F085516C0AD8A49BEFD0
:1044100029F08651410A3FE08651440A1BE086514B
:10442000420AD8B45EEF22F08651350AD8B427EF9D
:104430002BF08651360AD8B47CEF2BF08651370A20
:10444000D8B4E5EF2BF08651380AD8B443EF2CF0FE
:104450009BEF29F00798079A04017A0E826F96EC79
:104460000EF00401780E826F96EC0EF00401640EDB
:10447000826F96EC0EF00401550E826F96EC0EF0F2
:1044800047EF22F004014C0E826F96EC0EF0A0EC88
:104490000EF09DEF29F00788079A04017A0E826FCB
:1044A00096EC0EF00401410E826F96EC0EF00401C2
:1044B000610E826F96EC0EF03BEF22F00798078AB0
:1044C00004017A0E826F96EC0EF00401420E826FA8
:1044D00096EC0EF00401610E826F96EC0EF03BEF4D
:1044E00022F0010166677CEF22F067677CEF22F023
:1044F00068677CEF22F0696716D001014F6788EF8B
:1045000022F0506788EF22F0516788EF22F052675F
:104510000AD00101000E006F000E016F000E026F45
:10452000000E036F120011B80AD00101620E046F71
:10453000010E056F000E066F000E076F09D0010116
:10454000A70E046F020E056F000E066F000E076FB8
:1045500066C100F167C101F168C102F169C103F1EF
:1045600085EC2FF003BF25EF23F0119A119C010178
:10457000000E046FA80E056F550E066F020E076F32
:1045800066C100F167C101F168C102F169C103F1BF
:1045900066C18AF167C18BF168C18CF169C18DF187
:1045A00085EC2FF003BF0BD00101000E8A6FA80E1F
:1045B0008B6F550E8C6F020E8D6F118A119C0E0E33
:1045C00064EC0BF0E8CF18F10F0E64EC0BF0E8CFC1
:1045D00019F1100E64EC0BF0E8CF1AF1110E64EC37
:1045E0000BF0E8CF1BF1CEEC2EF08AC104F18BC1A9
:1045F00005F18CC106F18DC107F185EC2FF0078222
:1046000092EC2EF0CEEC2EF0079292EC2EF08AC1B6
:1046100000F18BC101F18CC102F18DC103F1079250
:1046200092EC2EF0CC0E046FE00E056F870E066F35
:10463000050E076F85EC2FF000C118F101C119F1CB
:1046400002C11AF103C11BF140D013AA2AEF23F0D3
:10465000138E139A119C119A0101800E006F1A0E8D
:10466000016F060E026F000E036F4FC104F150C1BF
:1046700005F151C106F152C107F185EC2FF003AFEE
:1046800005D09AEC30F0118C119A12000E0E64ECE9
:104690000BF0E8CF18F10F0E64EC0BF0E8CF19F136
:1046A000100E64EC0BF0E8CF1AF1110E64EC0BF075
:1046B000E8CF1BF14FC100F150C101F151C102F12E
:1046C00052C103F1078292EC2EF018C100F119C11A
:1046D00001F11AC102F11BC103F112000784BAC132
:1046E00066F1BBC167F1BCC168F1BDC169F14BC1E5
:1046F0004FF14CC150F14DC151F14EC152F157C172
:1047000059F158C15AF10794010166678FEF23F000
:1047100067678FEF23F068678FEF23F0696716D024
:1047200001014F679BEF23F050679BEF23F0516728
:104730009BEF23F052670AD00101000E006F000EBC
:10474000016F000E026F000E036F120011B80AD045
:104750000101620E046F010E056F000E066F000E60
:10476000076F09D00101A70E046F020E056F000E3E
:10477000066F000E076F66C100F167C101F168C1E5
:1047800002F169C103F185EC2FF003BF27EF24F09C
:104790000101000E046FA80E056F550E066F020E84
:1047A000076F66C100F167C101F168C102F169C11B
:1047B00003F166C18AF167C18BF168C18CF169C1EF
:1047C0008DF185EC2FF003BF09D00101000E8A6F37
:1047D000A80E8B6F550E8C6F020E8D6FCEEC2EF0E7
:1047E00000C104F101C105F102C106F103C107F1E5
:1047F000000E006FA00E016F980E026F7B0E036F0C
:10480000B6EC2FF000C118F101C119F102C11AF183
:1048100003C11BF1000E006FA00E016F980E026F16
:104820007B0E036F8AC104F18BC105F18CC106F1C7
:104830008DC107F1B6EC2FF018C104F119C105F1D3
:104840001AC106F11BC107F185EC2FF0120001011E
:10485000A80E006F610E016F000E026F000E036F55
:104860004FC104F150C105F151C106F152C107F128
:1048700085EC2FF003AF0AD00101A80E006F610E86
:10488000016F000E026F000E036F00D0C80E006FA4
:10489000AF0E016F000E026F000E036F4FC104F1E7
:1048A00050C105F151C106F152C107F196EC2FF04C
:1048B00012000401730E826F96EC0EF004012C0EB0
:1048C000826F96EC0EF0078462C166F163C167F1F6
:1048D00064C168F165C169F14BC14FF14CC150F140
:1048E0004DC151F14EC152F157C159F158C15AF160
:1048F00007947FEC24F0A0EC0EF09DEF29F066C148
:1049000000F167C101F168C102F169C103F1010160
:1049100023EC30F0E6EC2DF00401630E826F96EC90
:104920000EF004012C0E826F96EC0EF04FC100F1D8
:1049300050C101F151C102F152C103F1010123EC57
:1049400030F0E6EC2DF00401660E826F96EC0EF06E
:1049500004012C0E826F96EC0EF09AEC30F059C1E7
:1049600000F15AC101F1010123EC30F0E6EC2DF029
:104970000401740E826F96EC0EF012001082040196
:10498000530E826F96EC0EF004012C0E826F96ECA3
:104990000EF083C32AF184C32BF185C32CF186C3A7
:1049A0002DF187C32EF188C32FF189C330F18AC35B
:1049B00031F18BC332F18CC333F10101E8EC30F0FB
:1049C0005FEC30F000C166F101C167F102C168F12E
:1049D00003C169F18EC32AF18FC32BF190C32CF16F
:1049E00091C32DF192C32EF193C32FF194C330F1F3
:1049F00095C331F196C332F197C333F10101E8EC6D
:104A000030F05FEC30F000C14FF101C150F102C154
:104A100051F103C152F1DBEC30F099C32FF19AC38D
:104A200030F19BC331F19CC332F19DC333F10101DD
:104A3000E8EC30F05FEC30F000C159F101C15AF1FF
:104A40007FEC24F004012C0E826F96EC0EF039EF0F
:104A500025F0118E1CA002D01CAE108C1BBE02D003
:104A60001BA4108E03018251520A02E10F8201D071
:104A70000F928251750A02E1108401D01094825184
:104A8000550A02E1108601D010968351310A03E1E4
:104A90001382138402D01392139403018351660A84
:104AA00001E056D00401660E826F96EC0EF0040110
:104AB0002C0E826F96EC0EF06EEC23F023EC30F0AF
:104AC0002AC182F40401300E822796EC0EF02BC12D
:104AD00082F40401300E822796EC0EF02CC182F491
:104AE0000401300E822796EC0EF02DC182F40401F1
:104AF000300E822796EC0EF02EC182F40401300EA7
:104B0000822796EC0EF02FC182F40401300E82272A
:104B100096EC0EF030C182F40401300E822796EC40
:104B20000EF031C182F40401300E822796EC0EF0B3
:104B300032C182F40401300E822796EC0EF033C1AC
:104B400082F40401300E822796EC0EF09BEF29F0E0
:104B500011A003D011A401D01084078410B212EF69
:104B600026F010A4F6EF25F0BAC166F1BBC167F1DB
:104B7000BCC168F1BDC169F1BEC16AF1BFC16BF1D1
:104B8000C0C16CF1C1C16DF1C2C16EF1C3C16FF1A1
:104B9000C4C170F1C5C171F1C6C172F1C7C173F171
:104BA000C8C174F1C9C175F1CAC176F1CBC177F141
:104BB000CCC178F1CDC179F1CEC17AF1CFC17BF111
:104BC000D0C17CF1D1C17DF1D2C17EF1D3C17FF1E1
:104BD000D4C180F1D5C181F1D6C182F1D7C183F1B1
:104BE000D8C184F1D9C185F1FEEF25F062C166F12B
:104BF00063C167F164C168F165C169F1BAC186F149
:104C0000BBC187F1BCC188F1BDC189F14BC14FF176
:104C10004CC150F14DC151F14EC152F157C159F142
:104C200058C15AF107940FA034EF26F0010196679E
:104C300021EF26F0976721EF26F0986721EF26F005
:104C4000996725EF26F034EF26F071EC22F096C13B
:104C500004F197C105F198C106F199C107F185ECFE
:104C60002FF003BF61EF29F071EC22F00101000E7B
:104C7000046F000E056F010E066F000E076FB6EC95
:104C80002FF011A02AD011A228D023EC30F02967F0
:104C900001D005D004012D0E826F96EC0EF030C1CC
:104CA00082F40401300E822796EC0EF031C182F4BA
:104CB0000401300E822796EC0EF032C182F404011A
:104CC000300E822796EC0EF033C182F40401300ED0
:104CD000822796EC0EF0A0EC0EF012A8C5D0129828
:104CE0001DC01EF01E3A1E42070E1E1600011E5069
:104CF000000AD8B400EF27F000011E50010AD8B412
:104D00008CEF26F000011E50020AD8B48AEF26F07C
:104D100032EF27F032EF27F09AEC30F02DC001F19E
:104D20002EC000F1D89001330033D8900133003306
:104D30000101630E046F000E056F000E066F000E7A
:104D4000076FB6EC2FF0280E046F000E056F000EF3
:104D5000066F000E076F85EC2FF000C130F09AEC63
:104D600030F02BC001F1019F019D2CC000F1010129
:104D7000A40E046F000E056F000E066F000E076F85
:104D8000B6EC2FF000C12FF000C104F101C105F114
:104D900002C106F103C107F1640E006F000E016F3E
:104DA000000E026F000E036F85EC2FF0050E046FEE
:104DB000000E056F000E066F000E076FB6EC2FF0A9
:104DC00000C104F101C105F102C106F103C107F1FF
:104DD0009AEC30F030C000F185EC2FF000C131F0DA
:104DE00031C0E8FF050F305C03E78A8432EF27F01B
:104DF00031C0E8FF0A0F305C01E68A9432EF27F0F9
:104E000000C124F101C125F102C126F103C127F13E
:104E10009AEC30F0A0EC30F01D501F0BE8CF00F101
:104E20000101640E046F000E056F000E066F000E88
:104E3000076F96EC2FF024C104F125C105F126C1BE
:104E400006F127C107F185EC2FF003BF02D08A9449
:104E500001D08A8424C100F125C101F126C102F1EB
:104E600027C103F19DEF29F000C124F101C125F113
:104E700002C126F103C127F110AE4DD0109E00C132
:104E800008F101C109F102C10AF103C10BF123ECE0
:104E900030F030C1E2F131C1E3F132C1E4F133C1AC
:104EA000E5F108C100F109C101F10AC102F10BC12C
:104EB00003F101016C0E046F070E056F000E066F03
:104EC000000E076F85EC2FF003BF04D00101550ED3
:104ED000E66F1CD008C100F109C101F10AC102F15D
:104EE0000BC103F10101A40E046F060E056F000E45
:104EF000066F000E076F85EC2FF003BF04D0010191
:104F00007F0EE66F03D00101FF0EE66F1F8E11AE1C
:104F100061EF29F0119E24C100F125C101F126C1E4
:104F200002F127C103F111A005D011A203D00FB0E7
:104F300061EF29F010A4A4EF27F00401750E826F31
:104F400096EC0EF0A9EF27F00401720E826F96EC3A
:104F50000EF004012C0E826F96EC0EF023EC30F074
:104F60002967B8EF27F00401200E826FBBEF27F00E
:104F700004012D0E826F96EC0EF030C182F4040114
:104F8000300E822796EC0EF031C182F40401300E0F
:104F9000822796EC0EF004012E0E826F96EC0EF036
:104FA00032C182F40401300E822796EC0EF033C138
:104FB00082F40401300E822796EC0EF004016D0E8F
:104FC000826F96EC0EF004012C0E826F96EC0EF0C0
:104FD0004FC100F150C101F151C102F152C103F1C1
:104FE000010123EC30F0E6EC2DF00401480E826F55
:104FF00096EC0EF004017A0E826F96EC0EF004012E
:105000002C0E826F96EC0EF066C100F167C101F1C3
:1050100068C102F169C103F1010123EC30F0E6EC53
:105020002DF00401630E826F96EC0EF004012C0E3D
:10503000826F96EC0EF066C100F167C101F168C1A4
:1050400002F169C103F101010A0E046F000E056F40
:10505000000E066F000E076F96EC2FF0000E046F27
:10506000120E056F000E066F000E076FB6EC2FF0E4
:1050700023EC30F02AC182F40401300E822796EC32
:105080000EF02BC182F40401300E822796EC0EF054
:105090002CC182F40401300E822796EC0EF02DC153
:1050A00082F40401300E822796EC0EF02EC182F4B9
:1050B0000401300E822796EC0EF02FC182F4040119
:1050C000300E822796EC0EF030C182F40401300ECF
:1050D000822796EC0EF004012E0E826F96EC0EF0F5
:1050E00031C182F40401300E822796EC0EF032C1F9
:1050F00082F40401300E822796EC0EF033C182F464
:105100000401300E822796EC0EF00401730E826FBC
:1051100096EC0EF004012C0E826F96EC0EF09AECD9
:1051200030F059C100F15AC101F1C7EC2AF013A2C5
:10513000E9EF28F004012C0E826F96EC0EF086C188
:1051400066F187C167F188C168F189C169F171ECC5
:1051500022F00101000E046F000E056F010E066FB4
:10516000000E076FB6EC2FF023EC30F02967BEEF8E
:1051700028F00401200E826FC1EF28F004012D0EEB
:10518000826F96EC0EF030C182F40401300E82275B
:1051900096EC0EF031C182F40401300E822796ECB9
:1051A0000EF004012E0E826F96EC0EF032C182F4E6
:1051B0000401300E822796EC0EF033C182F4040114
:1051C000300E822796EC0EF004016D0E826F96EC85
:1051D0000EF013A410EF29F004012C0E826F96EC50
:1051E0000EF013ACFEEF28F00401500E826F96EC27
:1051F0000EF0139C1398139A10EF29F013AE0BEFD7
:1052000029F00401460E826F96EC0EF0139E13985F
:10521000139A10EF29F00401530E826F96EC0EF0F2
:1052200037B027EF29F004012C0E826F96EC0EF0B8
:105230008BB022EF29F00401440E826F96EC0EF041
:1052400027EF29F00401530E826F96EC0EF00FB297
:105250002DEF29F00FA05FEF29F004012C0E826FD3
:1052600096EC0EF0200EF86EF76AF66A040109005B
:10527000F5CF82F496EC0EF00900F5CF82F496ECAF
:105280000EF00900F5CF82F496EC0EF00900F5CF90
:1052900082F496EC0EF00900F5CF82F496EC0EF055
:1052A0000900F5CF82F496EC0EF00900F5CF82F4F8
:1052B00096EC0EF00900F5CF82F496EC0EF0A0EC1F
:1052C0000EF00F90109E12989DEF29F00401630ECE
:1052D000826F96EC0EF004012C0E826F96EC0EF0AD
:1052E000A3EC29F004012C0E826F96EC0EF016EC64
:1052F0002AF004012C0E826F96EC0EF092EC2AF04C
:1053000004012C0E826F96EC0EF00101F80E006F76
:10531000CD0E016F660E026F030E036FB8EC29F01D
:1053200004012C0E826F96EC0EF0A8EC2AF0A0EC93
:105330000EF09DEF29F0A0EC0EF00301C26B079078
:105340001092ACEF2CF0D8900E0E64EC0BF0E8CF7E
:1053500000F10F0E64EC0BF0E8CF01F1100E64ECDD
:105360000BF0E8CF02F1110E64EC0BF0E8CF03F183
:105370000101000E046F000E056F010E066F000E96
:10538000076FB6EC2FF023EC30F02AC182F4040151
:10539000300E822796EC0EF02BC182F40401300E01
:1053A000822796EC0EF02CC182F40401300E822785
:1053B00096EC0EF02DC182F40401300E822796EC9B
:1053C0000EF02EC182F40401300E822796EC0EF00E
:1053D0002FC182F40401300E822796EC0EF030C10A
:1053E00082F40401300E822796EC0EF031C182F473
:1053F0000401300E822796EC0EF004012E0E826F0F
:1054000096EC0EF032C182F40401300E822796EC45
:105410000EF033C182F40401300E822796EC0EF0B8
:1054200004016D0E826F96EC0EF01200120E64EC09
:105430000BF0E8CF00F1130E64EC0BF0E8CF01F1B4
:10544000140E64EC0BF0E8CF02F1150E64EC0BF0D7
:10545000E8CF03F101010A0E046F000E056F000E84
:10546000066F000E076F96EC2FF0000E046F120E01
:10547000056F000E066F000E076FB6EC2FF023ECE1
:1054800030F02AC182F40401300E822796EC0EF02F
:105490002BC182F40401300E822796EC0EF02CC151
:1054A00082F40401300E822796EC0EF02DC182F4B6
:1054B0000401300E822796EC0EF02EC182F4040116
:1054C000300E822796EC0EF02FC182F40401300ECC
:1054D000822796EC0EF030C182F40401300E822750
:1054E00096EC0EF004012E0E826F96EC0EF031C198
:1054F00082F40401300E822796EC0EF032C182F461
:105500000401300E822796EC0EF033C182F40401C0
:10551000300E822796EC0EF00401730E826F96EC2B
:105520000EF012000A0E64EC0BF0E8CF00F10B0E47
:1055300064EC0BF0E8CF01F10C0E64EC0BF0E8CF5B
:1055400002F10D0E64EC0BF0E8CF03F1C7EF2AF087
:10555000060E64EC0BF0E8CF00F1070E64EC0BF0E4
:10556000E8CF01F1080E64EC0BF0E8CF02F1090E70
:1055700064EC0BF0E8CF03F1C7EF2AF001019AECDD
:1055800030F0078457C100F158C101F107940101BF
:10559000E80E046F800E056F000E066F000E076F99
:1055A00096EC2FF0000E046F040E056F000E066FD0
:1055B000000E076FB6EC2FF0880E046F130E056F08
:1055C000000E066F000E076F85EC2FF00A0E046FB9
:1055D000000E056F000E066F000E076FB6EC2FF081
:1055E00023EC30F001012967FBEF2AF00401200EC3
:1055F000826FFEEF2AF004012D0E826F96EC0EF002
:1056000030C182F40401300E822796EC0EF031C1D5
:1056100082F40401300E822796EC0EF032C182F43F
:105620000401300E822796EC0EF004012E0E826FDC
:1056300096EC0EF033C182F40401300E822796EC12
:105640000EF00401430E826F96EC0EF0120087C339
:105650002AF188C32BF189C32CF18AC32DF18BC3A6
:105660002EF18CC32FF18DC330F18EC331F190C375
:1056700032F191C333F10101296BE8EC30F05FECBA
:1056800030F00101000E046F000E056F010E066F71
:10569000000E076F96EC2FF00E0E0C6E00C10BF093
:1056A0004DEC0BF00F0E0C6E01C10BF04DEC0BF03E
:1056B000100E0C6E02C10BF04DEC0BF0110E0C6EC7
:1056C00003C10BF04DEC0BF004017A0E826F96ECE7
:1056D0000EF004012C0E826F96EC0EF00401350ED4
:1056E000826F96EC0EF004012C0E826F96EC0EF099
:1056F000A3EC29F047EF22F087C32AF188C32BF1EE
:1057000089C32CF18AC32DF18BC32EF18CC32FF1E9
:105710008DC330F18EC331F190C332F191C333F1B7
:105720000101296BE8EC30F05FEC30F0880E046F7B
:10573000130E056F000E066F000E076F8AEC2FF038
:10574000000E046F040E056F000E066F000E076F4B
:1057500096EC2FF00101E80E046F800E056F000E2D
:10576000066F000E076FB6EC2FF00A0E0C6E00C12C
:105770000BF04DEC0BF00B0E0C6E01C10BF04DEC71
:105780000BF00C0E0C6E02C10BF04DEC0BF00D0E7D
:105790000C6E03C10BF04DEC0BF004017A0E826F1E
:1057A00096EC0EF004012C0E826F96EC0EF00401C4
:1057B000360E826F96EC0EF004012C0E826F96EC82
:1057C0000EF092EC2AF047EF22F087C32AF188C34B
:1057D0002BF189C32CF18AC32DF18BC32EF18CC31D
:1057E0002FF18DC330F18FC331F190C332F191C3EA
:1057F00033F10101E8EC30F05FEC30F0000E046FA3
:10580000120E056F000E066F000E076F96EC2FF05C
:1058100001010A0E046F000E056F000E066F000EE8
:10582000076FB6EC2FF0120E0C6E00C10BF04DECB2
:105830000BF0130E0C6E01C10BF04DEC0BF0140EBF
:105840000C6E02C10BF04DEC0BF0150E0C6E03C18B
:105850000BF04DEC0BF004017A0E826F96EC0EF01B
:1058600004012C0E826F96EC0EF00401370E826F4D
:1058700096EC0EF004012C0E826F96EC0EF016ECF6
:105880002AF047EF22F087C32AF188C32BF189C39E
:105890002CF18AC32DF18BC32EF18CC32FF18DC354
:1058A00030F18EC331F190C332F191C333F1010174
:1058B000296BE8EC30F05FEC30F0880E046F130ECB
:1058C000056F000E066F000E076F8AEC2FF0000EBA
:1058D000046F040E056F000E066F000E076F96EC46
:1058E0002FF00101E80E046F800E056F000E066FA9
:1058F000000E076FB6EC2FF0060E0C6E00C10BF019
:105900004DEC0BF0070E0C6E01C10BF04DEC0BF0E3
:10591000080E0C6E02C10BF04DEC0BF0090E0C6E74
:1059200003C10BF04DEC0BF004017A0E826F96EC84
:105930000EF004012C0E826F96EC0EF00401380E6E
:10594000826F96EC0EF004012C0E826F96EC0EF036
:10595000A8EC2AF047EF22F007A81FEF2DF0010175
:10596000800E006F1A0E016F060E026F000E036F9D
:105970004BC104F14CC105F14DC106F14EC107F117
:1059800085EC2FF003BF65EF2DF0E0EC2DF04BC15F
:1059900000F14CC101F14DC102F14EC103F107828A
:1059A00092EC2EF018C104F119C105F11AC106F1EB
:1059B0001BC107F1F80E006FCD0E016F660E026F6E
:1059C000030E036F85EC2FF00E0E0C6E00C10BF072
:1059D0004DEC0BF00F0E0C6E01C10BF04DEC0BF00B
:1059E000100E0C6E02C10BF04DEC0BF0110E0C6E94
:1059F00003C10BF04DEC0BF0078401019AEC30F081
:105A000057C100F158C101F107940A0E0C6E00C194
:105A10000BF04DEC0BF00B0E0C6E01C10BF04DECCE
:105A20000BF00C0E0C6E02C10BF04DEC0BF00D0EDA
:105A30000C6E03C10BF04DEC0BF065EF2DF007AAD7
:105A400065EF2DF0078401019AEC30F057C100F1A9
:105A500058C101F10794060E0C6E00C10BF04DEC1D
:105A60000BF0070E0C6E01C10BF04DEC0BF0080EA5
:105A70000C6E02C10BF04DEC0BF0090E0C6E03C165
:105A80000BF04DEC0BF0078462C100F163C101F132
:105A900064C102F165C103F10794120E0C6E00C1DE
:105AA0000BF04DEC0BF0130E0C6E01C10BF04DEC36
:105AB0000BF0140E0C6E02C10BF04DEC0BF0150E3A
:105AC0000C6E03C10BF04DEC0BF00798079A040124
:105AD000805181197F0B0DE09EA8FED714EE00F0D7
:105AE00081517F0BE126E750812B0F01AD6E67EFEF
:105AF0002DF005012F51000AD8B4A8EF2DF081BA7E
:105B00008DEF2DF015B2A8EF2DF005012F51010AF0
:105B1000D8B4A6EF2DF09FEF2DF005012F51000A0C
:105B2000D8B45FEF38F005012F51010AD8B4A6EFC1
:105B30002DF000011650050AD8B45FEF38F081B897
:105B4000A8EF2DF0E3EC31F0E1EC32F0F8EC37F0B7
:105B5000C4EF0DF018C100F119C101F11AC102F131
:105B60001BC103F1000E046F000E056F010E066FDE
:105B7000000E076FB6EC2FF029A1D5EF2DF02051C4
:105B8000D8B4D5EF2DF018C100F119C101F11AC137
:105B900002F11BC103F1000E046F000E056F0A0E27
:105BA000066F000E076FB6EC2FF0120001010451D2
:105BB000001305510113065102130751031312007C
:105BC0000101186B196B1A6B1B6B12002AC182F44E
:105BD0000401300E822796EC0EF02BC182F40401F2
:105BE000300E822796EC0EF02CC182F40401300EA8
:105BF000822796EC0EF02DC182F40401300E82272C
:105C000096EC0EF02EC182F40401300E822796EC41
:105C10000EF02FC182F40401300E822796EC0EF0B4
:105C200030C182F40401300E822796EC0EF031C1AF
:105C300082F40401300E822796EC0EF032C182F419
:105C40000401300E822796EC0EF033C182F4040179
:105C5000300E822796EC0EF012002FC182F4040160
:105C6000300E822796EC0EF030C182F40401300E23
:105C7000822796EC0EF031C182F40401300E8227A7
:105C800096EC0EF032C182F40401300E822796ECBD
:105C90000EF033C182F40401300E822796EC0EF030
:105CA0001200060E216E060E226E060E236E212EA7
:105CB00057EF2EF0222E57EF2EF0232E57EF2EF017
:105CC0008B84020E216E020E226E020E236E212E96
:105CD00067EF2EF0222E67EF2EF0232E67EF2EF0C7
:105CE0008B941200FF0E226E22C023F0030E216E51
:105CF0008B84212E78EF2EF0030E216E232E78EF69
:105D00002EF08B9422C023F0030E216E212E86EFFD
:105D10002EF0030E216E233E86EF2EF0222E74EF1E
:105D20002EF012000101005305E1015303E102537B
:105D300001E1002B55EC2FF09AEC30F03951006F57
:105D40003A51016F420E046F4B0E056F000E066F45
:105D5000000E076F96EC2FF000C104F101C105F1B0
:105D600002C106F103C107F118C100F119C101F127
:105D70001AC102F11BC103F107B2C3EF2EF08AEC86
:105D80002FF0C5EF2EF085EC2FF000C118F101C106
:105D900019F102C11AF103C11BF112009AEC30F0A3
:105DA00059C100F15AC101F1060E64EC0BF0E8CFC5
:105DB00004F1070E64EC0BF0E8CF05F1080E64EC7B
:105DC0000BF0E8CF06F1090E64EC0BF0E8CF07F119
:105DD00085EC2FF000C124F101C125F102C126F1AB
:105DE00003C127F1290E046F000E056F000E066F28
:105DF000000E076F96EC2FF0EE0E046F430E056F4A
:105E0000000E066F000E076F8AEC2FF024C104F11C
:105E100025C105F126C106F127C107F196EC2FF047
:105E200000C11CF101C11DF102C11EF103C11FF12E
:105E3000120E64EC0BF0E8CF04F1130E64EC0BF0DF
:105E4000E8CF05F1140E64EC0BF0E8CF06F1150E67
:105E500064EC0BF0E8CF07F10D0E006F000E016F40
:105E6000000E026F000E036F96EC2FF0180E046FF9
:105E7000000E056F000E066F000E076FB6EC2FF0D8
:105E80001CC104F11DC105F11EC106F11FC107F1BE
:105E90008AEC2FF06A0E046F2A0E056F000E066F53
:105EA000000E076F85EC2FF01200BF0EFA6E200E69
:105EB0003A6F396BD8900037013702370337D8B0C3
:105EC00066EF2FF03A2F5BEF2FF039073A070353B5
:105ED000D8B412000331070B80093F6F03390F0B51
:105EE000010F396F80EC5FF0406F390580EC5FF097
:105EF000405D405F396B3F33D8B0392739333FA914
:105F00007BEF2FF04051392712000101BFEC30F038
:105F1000D8B01200010103510719346F82EC30F040
:105F2000D8900751031934AF800F12000101346B70
:105F3000A6EC30F0D8A0BCEC30F0D8B0120091EC58
:105F400030F09AEC30F01F0E366FD2EC30F00B359B
:105F5000D8B082EC30F0D8A00335D8B01200362F7C
:105F6000A5EF2FF034B1A9EC30F012000101346B31
:105F700004510511061107110008D8A0A6EC30F055
:105F8000D8A0BCEC30F0D8B01200086B096B0A6BDB
:105F90000B6BD2EC30F01F0E366FD2EC30F00751A5
:105FA0000B5DD8A4E0EF2FF006510A5DD8A4E0EF16
:105FB0002FF00551095DD8A4E0EF2FF00451085DE2
:105FC000D8A0F3EF2FF00451085F0551D8A0053D8C
:105FD000095F0651D8A0063D0A5F0751D8A0073DCA
:105FE0000B5FD8900081362FCDEF2FF034B1A9ECA4
:105FF00030F0346BA6EC30F0D890D6EC30F007518E
:106000000B5DD8A410EF30F006510A5DD8A410EF54
:1060100030F00551095DD8A410EF30F00451085D4F
:10602000D8A01FEF30F0003F1FEF30F0013F1FEF0F
:1060300030F0023F1FEF30F0032BD8B4120034B120
:10604000A9EC30F012000101346BA6EC30F0D8B0AE
:106050001200DBEC30F0200E366F003701370237CC
:10606000033711EE33F00A0E376FE7360A0EE75C9E
:10607000D8B0E76EE552372F35EF30F0362F2DEFE1
:1060800030F034B12981D8901200DBEC30F0200ED2
:10609000366F003701370237033711EE33F00A0E3F
:1060A000376FE7360A0EE75CD8B0E76EE552372F58
:1060B00051EF30F0362F49EF30F0D8901200010147
:1060C0000A0E346F200E366F11EE29F03451376FFF
:1060D0000A0ED890E652D8B0E726E732372F6AEF9B
:1060E00030F00333023301330033362F64EF30F0E6
:1060F000E750FF0FD8A00335D8B0120029B1A9ECA2
:1061000030F01200045100270551D8B0053D012799
:106110000651D8B0063D02270751D8B0073D0327E6
:1061200012000051086F0151096F02510A6F0351AB
:106130000B6F12000101006B016B026B036B12000D
:106140000101046B056B066B076B12000335D8A0C9
:1061500012000351800B001F011F021F031F003F8D
:10616000B9EF30F0013FB9EF30F0023FB9EF30F056
:10617000032B342B032512000735D8A0120007513A
:10618000800B041F051F061F071F043FCFEF30F0D1
:10619000053FCFEF30F0063FCFEF30F0072B342B29
:1061A0000725120000370137023703370837093750
:1061B0000A370B3712000101296B2A6B2B6B2C6BF2
:1061C0002D6B2E6B2F6B306B316B326B336B120080
:1061D00001012A510F0B2A6F2B510F0B2B6F2C51E2
:1061E0000F0B2C6F2D510F0B2D6F2E510F0B2E6F90
:1061F0002F510F0B2F6F30510F0B306F31510F0B91
:10620000316F32510F0B326F33510F0B336F12005E
:1062100000C124F101C125F102C126F103C127F11A
:1062200004C100F105C101F106C102F107C103F18A
:1062300024C104F125C105F126C106F127C107F1EA
:10624000120010A806D08994000EC76E220EC66EEA
:1062500005D08984000EC76E220EC66E050EE82E8C
:10626000FED7120010A802D0898401D08994050EAF
:10627000E82EFED7120021EC31F09E96C69E000E4D
:10628000C96EFF0E9EB602D0E82EFCD79E96C69E23
:10629000000EC96EFF0E9EB602D0E82EFCD7C9CF05
:1062A000AFF59E96C69E000EC96EFF0E9EB602D03A
:1062B000E82EFCD7C9CFB0F59E96C69E000EC96EDB
:1062C000FF0E9EB602D0E82EFCD7C9CFB1F59E9640
:1062D000C69E000EC96EFF0E9EB602D0E82EFCD7F9
:1062E000C9CFB2F59E96C69E000EC96EFF0E9EB631
:1062F00002D0E82EFCD7C9CFB3F59E96C69E000EFD
:10630000C96EFF0E9EB602D0E82EFCD7C9CFB4F5F9
:106310009E96C69E000EC96EFF0E9EB602D0E82E57
:10632000FCD7C9CFB5F532EC31F0120021EC31F0D9
:106330009E96C69E800EC96EFF0E9EB602D0E82EB7
:10634000FCD79E96C69EAFC5C9FFFF0E9EB602D073
:10635000E82EFCD79E96C69EB0C5C9FFFF0E9EB61E
:1063600002D0E82EFCD79E96C69EB1C5C9FFFF0E8F
:106370009EB602D0E82EFCD79E96C69EB2C5C9FF37
:10638000FF0E9EB602D0E82EFCD79E96C69EB3C5E1
:10639000C9FFFF0E9EB602D0E82EFCD79E96C69E81
:1063A000B4C5C9FFFF0E9EB602D0E82EFCD79E965C
:1063B000C69EB5C5C9FFFF0E9EB602D0E82EFCD71B
:1063C00032EC31F0120021EC31F09E96C69E070EA1
:1063D000C96EFF0E9EB602D0E82EFCD79E96C69ED2
:1063E000000EC96EFF0E9EB602D0E82EFCD7C9CFB4
:1063F000AFF59E96C69E000EC96EFF0E9EB602D0E9
:10640000E82EFCD7C9CFB0F59E96C69E000EC96E89
:10641000FF0E9EB602D0E82EFCD7C9CFB1F59E96EE
:10642000C69E000EC96EFF0E9EB602D0E82EFCD7A7
:10643000C9CFB2F532EC31F021EC31F09E96C69E18
:1064400025C0C9FFFF0E9EB602D0E82EFCD79E964F
:10645000C69E000EC96EFF0E9EB602D0E82EFCD777
:10646000C9CFB6F532EC31F0120021EC31F09E9636
:10647000C69E870EC96EFF0E9EB602D0E82EFCD7D0
:106480009E96C69EAFC5C9FFFF0E9EB602D0E82EEF
:10649000FCD79E96C69EB0C5C9FFFF0E9EB602D021
:1064A000E82EFCD79E96C69EB1C5C9FFFF0E9EB6CC
:1064B00002D0E82EFCD79E96C69EB2C5C9FFFF0E3D
:1064C0009EB602D0E82EFCD732EC31F021EC31F050
:1064D0009E96C69E26C0C9FFFF0E9EB602D0E82E2D
:1064E000FCD79E96C69EB6C5C9FFFF0E9EB602D0CB
:1064F000E82EFCD732EC31F0120021EC31F09E9600
:10650000C69E870EC96EFF0E9EB602D0E82EFCD73F
:106510009E96C69E000EC96EFF0E9EB602D0E82E55
:10652000FCD79E96C69E800EC96EFF0E9EB602D008
:10653000E82EFCD79E96C69E800EC96EFF0E9EB6B4
:1065400002D0E82EFCD79E96C69E800EC96EFF0E26
:106550009EB602D0E82EFCD732EC31F0120021ECCE
:1065600031F09E96C69E870EC96EFF0E9EB602D073
:10657000E82EFCD79E96C69E000EC96EFF0E9EB6F4
:1065800002D0E82EFCD79E96C69E000EC96EFF0E66
:106590009EB602D0E82EFCD79E96C69E800EC96E8F
:1065A000FF0E9EB602D0E82EFCD79E96C69E800EA9
:1065B000C96EFF0E9EB602D0E82EFCD732EC31F049
:1065C000120010A817D021EC31F09E96C69E8F0EB7
:1065D000C96EFF0E9EB602D0E82EFCD79E96C69ED0
:1065E000000EC96EFF0E9EB602D0E82EFCD732EC2C
:1065F00031F01200E3EC31F0120010A82DD021ECA4
:1066000031F09E96C69E26C0C9FFFF0E9EB602D0F0
:10661000E82EFCD79E96C69E450EC96EFF0E9EB60E
:1066200002D0E82EFCD732EC31F021EC31F09E960E
:10663000C69E8F0EC96EFF0E9EB602D0E82EFCD706
:106640009E96C69E000EC96EFF0E9EB602D0E82E24
:10665000FCD732EC31F0120021EC31F09E96C69E50
:1066600026C0C9FFFF0E9EB602D0E82EFCD79E962C
:10667000C69E010EC96EFF0E9EB602D0E82EFCD754
:1066800032EC31F021EC31F09E96C69E910EC96E2F
:10669000FF0E9EB602D0E82EFCD79E96C69EA50E93
:1066A000C96EFF0E9EB602D0E82EFCD732EC31F058
:1066B000120021EC31F09E96C69E26C0C9FFFF0E47
:1066C0009EB602D0E82EFCD79E96C69E810EC96E5D
:1066D000FF0E9EB602D0E82EFCD732EC31F012004D
:1066E00021EC31F09E96C69E26C0C9FFFF0E9EB6D5
:1066F00002D0E82EFCD79E96C69E010EC96EFF0EF4
:106700009EB602D0E82EFCD732EC31F0120021EC1C
:1067100031F09E96C69E910EC96EFF0E9EB602D0B7
:10672000E82EFCD79E96C69EA50EC96EFF0E9EB69D
:1067300002D0E82EFCD732EC31F0120021EC31F01F
:106740009E96C69E910EC96EFF0E9EB602D0E82E92
:10675000FCD79E96C69E000EC96EFF0E9EB602D056
:10676000E82EFCD732EC31F012000501256B266BC8
:10677000276B286B899A400EC76E200EC66E9E96B8
:10678000C69E030EC96EFF0E9EB602D0E82EFCD741
:106790009E96C69E27C5C9FFFF0E9EB602D0E82E64
:1067A000FCD79E96C69E26C5C9FFFF0E9EB602D098
:1067B000E82EFCD79E96C69E25C5C9FFFF0E9EB645
:1067C00002D0E82EFCD79E96C69EC952FF0E9EB6FA
:1067D00002D0E82EFCD7898A0F01C950FF0A01E1D7
:1067E000120005012E51130A05E005012E51170A6A
:1067F0000CE012000501F00E256FFF0E266F0F0E44
:10680000276F000E286F0EEF34F00501F00E256F94
:10681000FF0E266FFF0E276F000E286F899A400E1D
:10682000C76E200EC66E9E96C69E030EC96EFF0EE4
:106830009EB602D0E82EFCD79E96C69E27C5C9FFFD
:10684000FF0E9EB602D0E82EFCD79E96C69E26C5A9
:10685000C9FFFF0E9EB602D0E82EFCD79E96C69EBC
:1068600025C5C9FFFF0E9EB602D0E82EFCD79E9626
:10687000C69EC952FF0E9EB602D0E82EFCD7898A6A
:106880000F01C950FF0A1DE005012E51130A05E052
:1068900005012E51170A0BE012000501000E256FAD
:1068A000000E266F100E276F000E286F12000501D4
:1068B000000E256F000E266F000E276F010E286F49
:1068C00012000501256B266B276B286B05012E51E5
:1068D000130A05E005012E51170A0CE0120005010C
:1068E000000E216F000E226F080E236F000E246F22
:1068F00083EF34F00501000E216F000E226F800E31
:10690000236F000E246F21C500F122C501F123C5BC
:1069100002F124C503F125C504F126C505F127C5FB
:1069200006F128C507F1D6EC2DF000C125F501C10F
:1069300026F502C127F503C128F5899A400EC76ED6
:10694000200EC66E9E96C69E030EC96EFF0E9EB6A4
:1069500002D0E82EFCD79E96C69E27C5C9FFFF0E23
:106960009EB602D0E82EFCD79E96C69E26C5C9FFCD
:10697000FF0E9EB602D0E82EFCD79E96C69E25C579
:10698000C9FFFF0E9EB602D0E82EFCD79E96C69E8B
:10699000C952FF0E9EB602D0E82EFCD7898AC95094
:1069A000FF0A08E104C125F505C126F506C127F552
:1069B00007C128F5D890050124332333223321332E
:1069C0002151F00B216F05012167EEEF34F02267B2
:1069D000EEEF34F02367EEEF34F0246783EF34F00A
:1069E0000501100E2527E86A2623E86A2723E86AAE
:1069F00028231200E86A05012E51130A06E005015A
:106A00002E51170A0BE0020E120005012851000A50
:106A100003E12751F00B07E0010E12000501285198
:106A2000000A01E0010E120029C500F12AC501F19A
:106A30002BC502F12CC503F125C504F126C505F1CE
:106A400027C506F128C507F185EC2FF003BF12001A
:106A5000FAEC34F0D8A48CEF35F0899A400EC76E6A
:106A6000200EC66E9E96C69E060EC96EFF0E9EB680
:106A700002D0E82EFCD7898A899A9E96C69E020E7D
:106A8000C96EFF0E9EB602D0E82EFCD79E96C69E1B
:106A900027C5C9FFFF0E9EB602D0E82EFCD79E96F2
:106AA000C69E26C5C9FFFF0E9EB602D0E82EFCD7B3
:106AB0009E96C69E25C5C9FFFF0E9EB602D0E82E43
:106AC000FCD79E96C69E000EC96EFF0E9EB602D0E3
:106AD000E82EFCD7898A899A9E96C69E050EC96EB5
:106AE000FF0E9EB602D0E82EFCD79E96C69EC952D7
:106AF000FF0E9EB602D0E82EFCD7C9B075EF35F078
:106B0000898A0501100E2527E86A2623E86A2723CB
:106B1000E86A282314EF35F01200899A400EC76EF8
:106B2000200EC66E9E96C69E060EC96EFF0E9EB6BF
:106B300002D0E82EFCD7898A899A9E96C69EC70EF7
:106B4000C96EFF0E9EB602D0E82EFCD7898A0501D9
:106B5000256B266B276B286B1200899A400EC76E37
:106B6000200EC66E9E96C69E050EC96EFF0E9EB680
:106B700002D0E82EFCD79E96C69EC952FF0E9EB646
:106B800002D0E82EFCD7C9CF37F5898A1200899A3E
:106B9000400EC76E200EC66E9E96C69EB90EC96E7A
:106BA000FF0E9EB602D0E82EFCD7898A1200899A81
:106BB000400EC76E200EC66E9E96C69EAB0EC96E68
:106BC000FF0E9EB602D0E82EFCD7898AFF0EE82E73
:106BD000FED71200FAEC34F0D8A41200899A400EC5
:106BE000C76E200EC66E9E96C69E030EC96EFF0E21
:106BF0009EB602D0E82EFCD79E96C69E27C5C9FF3A
:106C0000FF0E9EB602D0E82EFCD79E96C69E26C5E5
:106C1000C9FFFF0E9EB602D0E82EFCD79E96C69EF8
:106C200025C5C9FFFF0E9EB602D0E82EFCD79E9662
:106C3000C69EC952FF0E9EB602D0E82EFCD7898AA6
:106C40000F01C950FF0AD8A469EF37F00501FE0E05
:106C5000376F0501FF0E536FFF0E546FFF0E556F18
:106C6000FF0E566F15A6379915863BEC31F0AFC570
:106C700038F5B0C539F5B1C53AF5B2C53BF5B3C580
:106C80003CF5B4C53DF5B5C53EF50784BAC166F11E
:106C9000BBC167F1BCC168F1BDC169F14BC14FF126
:106CA0004CC150F14DC151F14EC152F157C159F192
:106CB00058C15AF100011650010AD8B46EEF36F0EF
:106CC00000011650020AD8B493EF36F000011650B6
:106CD000040AD8B4B8EF36F069EF37F00501476B16
:106CE000486B496B4A6B05014B6B4C6B4D6B4E6BA4
:106CF00005014F6B506B516B526B8BA0379B71EC46
:106D000022F000C1DAF101C1DBF102C1DCF103C103
:106D1000DDF100C13FF501C140F502C141F503C1FC
:106D200042F5D7EF36F00501476B486B496B4A6B6C
:106D300005014B6B4C6B4D6B4E6B05014F6B506BF4
:106D4000516B526B71EC22F000C1DAF101C1DBF141
:106D500002C1DCF103C1DDF16EEC23F000C147F5A7
:106D600001C148F502C149F503C14AF569EF37F0A1
:106D7000379BDAC13FF5DBC140F5DCC141F5DDC130
:106D800042F571EC22F000C14BF501C14CF502C196
:106D90004DF503C14EF56EEC23F000C14FF501C176
:106DA00050F502C151F503C152F5D7EF36F0050198
:106DB0006167E2EF36F06267E2EF36F06367E2EFB9
:106DC00036F06467E6EF36F0FBEF36F0DAC100F13B
:106DD000DBC101F1DCC102F1DDC103F161C504F1E8
:106DE00062C505F163C506F164C507F185EC2FF0B6
:106DF00003BF69EF37F059C143F55AC144F5B9C52E
:106E000045F50501110E326F899A400EC76E200EAE
:106E1000C66E9E96C69E060EC96EFF0E9EB602D028
:106E2000E82EFCD7898A899A9E96C69E020EC96E64
:106E3000FF0E9EB602D0E82EFCD79E96C69E27C5B2
:106E4000C9FFFF0E9EB602D0E82EFCD79E96C69EC6
:106E500026C5C9FFFF0E9EB602D0E82EFCD79E962F
:106E6000C69E25C5C9FFFF0E9EB602D0E82EFCD7F0
:106E700025EE37F0322F02D049EF37F09E96C69EAE
:106E8000DECFC9FFFF0E9EB602D0E82EFCD73AEF48
:106E900037F0898A899A9E96C69E050EC96EFF0EA6
:106EA0009EB602D0E82EFCD79E96C69EC952FF0E13
:106EB0009EB602D0E82EFCD7C9B054EF37F0898ACD
:106EC0000501100E2527E86A2623E86A2723E86AC9
:106ED000282315900794120021C500F122C501F165
:106EE00023C502F124C503F1899A400EC76E200E16
:106EF000C66E9E96C69E0B0EC96EFF0E9EB602D043
:106F0000E82EFCD79E96C69E02C1C9FFFF0E9EB614
:106F100002D0E82EFCD79E96C69E01C1C9FFFF0E87
:106F20009EB602D0E82EFCD79E96C69E00C1C9FF31
:106F3000FF0E9EB602D0E82EFCD79E96C69EC95282
:106F4000FF0E9EB602D0E82EFCD725EE37F00501E5
:106F5000100E326F9E96C69EC952FF0E9EB602D08C
:106F6000E82EFCD7C9CFDEFF322FAAEF37F0898A8F
:106F70001200899A400EC76E200EC66E9E96C69E5F
:106F8000900EC96EFF0E9EB602D0E82EFCD79E96DC
:106F9000C69E000EC96EFF0E9EB602D0E82EFCD72C
:106FA0009E96C69E000EC96EFF0E9EB602D0E82EBB
:106FB000FCD79E96C69E000EC96EFF0E9EB602D0EE
:106FC000E82EFCD79E96C69EC952FF0E9EB602D0F2
:106FD000E82EFCD7C9CF2DF59E96C69EC952FF0E4E
:106FE0009EB602D0E82EFCD7C9CF2EF5898A1200B2
:106FF0003BEC31F005012F51010A5FE005012F51F3
:10700000020A16E005012F51030A19E005012F516C
:10701000040A24E005012F51050A2BE005012F5138
:10702000060A39E005012F51070A3FE05DEF38F00D
:10703000602F5BEF38F05FC560F55DEF38F0B0C5ED
:1070400000F101010F0E001701010051000A35E0A7
:1070500001010051050A31E05BEF38F0B0C500F1E5
:1070600001010F0E001701010051000A26E05BEF3D
:1070700038F00501B051000A20E00501B051150AB1
:107080001CE00501B051300A18E00501B051450A75
:1070900014E05BEF38F00501B051000A0EE0050185
:1070A000B051300A0AE05BEF38F00501B051000A38
:1070B00004E05BEF38F015901200158012008B9001
:1070C00051EC2EF0B9C5E8FFD70802E351EC2EF0E1
:1070D000B9C5E8FFC80802E351EC2EF0B9C5E8FFD6
:1070E000B90802E351EC2EF0B9C5E8FFAA0802E3A3
:1070F00051EC2EF0B9C5E8FF9B0802E351EC2EF0ED
:10710000C7EC35F0F29CF29E8B94C69AC2909482A2
:10711000948C720ED36ED3A4FED789968A909390E6
:10712000F29AF2949D909E909D929E92F298F29285
:10713000E1EC32F0FF0EE8CF00F0E82EFED7002E93
:10714000FCD7F290F286815081A8A9EF38F0F29E28
:107150000300700ED36EF296F2901584038072ECE9
:067160002EF09AEF0BF087
:10BF0000E844F926000C160C2B0C3F0C520C640C68
:10BF1000760C860C960CA50CB30CC10CCF0CDC0C6B
:06BF2000E80CF40C000C1B
:0200000400F00A
:0100C800FE39
:00000001FF
